:020000040000FA
:040800004DEF0BF0BD
:1008100003B276EF05F0F2B494EF05F09EB09CEFD2
:1008200005F09EB2A4EF05F0F2A81AEF04F0F2B2C0
:1008300025EF04F0F2A620EF04F0F2B022EF04F06E
:10084000FCEF0AF0F296F290FF00CD90F2929EA09B
:100850002FEF04F00101533F2FEF04F0542BAEC1F2
:10086000B2F1AFC1B3F1B0C1B4F1B1C1B5F1AAC138
:10087000AEF1ABC1AFF1ACC1B0F1ADC1B1F1A6C148
:10088000AAF1A7C1ABF1A8C1ACF1A9C1ADF1A2C158
:10089000A6F1A3C1A7F1A4C1A8F1A5C1A9F19EC168
:1008A000A2F19FC1A3F1A0C1A4F1A1C1A5F19AC178
:1008B0009EF19BC19FF19CC1A0F19DC1A1F196C188
:1008C0009AF197C19BF198C19CF199C19DF1CECF4E
:1008D00096F1CFCF97F153C198F154C199F1CF6AF6
:1008E000CE6A0101536B546B9E90CD800FBC0F8E6E
:1008F0000FBA7EEF04F00F8AFCEF0AF00F8C0FBEE8
:10090000BAEF04F096C19AF197C19BF198C19CF19E
:1009100099C19DF19AC19EF19BC19FF19CC1A0F12B
:100920009DC1A1F19EC1A2F19FC1A3F1A0C1A4F1FB
:10093000A1C1A5F1A2C1A6F1A3C1A7F1A4C1A8F1CB
:10094000A5C1A9F1A6C1AAF1A7C1ABF1A8C1ACF19B
:10095000A9C1ADF1AAC1AEF1ABC1AFF1ACC1B0F16B
:10096000ADC1B1F1AEC1B2F1AFC1B3F1B0C1B4F13B
:10097000B1C1B5F101015E6B5F6B606B616B96514C
:100980005E2797515F2398516023995161239A51B3
:100990005E279B515F239C5160239D5161239E5193
:1009A0005E279F515F23A0516023A1516123A25173
:1009B0005E27A3515F23A4516023A5516123A65153
:1009C0005E27A7515F23A8516023A9516123AA5133
:1009D0005E27AB515F23AC516023AD516123AE5113
:1009E0005E27AF515F23B0516023B1516123B251F3
:1009F0005E27B3515F23B4516023B5516123D89072
:100A00000101613360335F335E33D890010161339C
:100A100060335F335E33D8900101613360335F33FD
:100A20005E3300C10CF101C10DF102C10EF103C131
:100A30000FF104C110F105C111F106C112F107C196
:100A400013F108C114F109C115F10AC116F10BC166
:100A500017F134C135F111B839EF05F00101620E1B
:100A6000046F010E056F000E066F000E076F42EF58
:100A700005F00101A70E046F020E056F000E066F50
:100A8000000E076F5EC100F15FC101F160C102F1AC
:100A900061C103F1FEEC2BF003BF04D019BE02D0FC
:100AA00019A0108C11A05AEF05F010BA5AEF05F0FA
:100AB0000F80108A0CC100F10DC101F10EC102F1CD
:100AC0000FC103F110C104F111C105F112C106F10A
:100AD00013C107F114C108F115C109F116C10AF1DA
:100AE00017C10BF135C134F1FCEF0AF00392ABB240
:100AF000AB98AB88030103EE00F080517F0BE92631
:100B000004C0EFFF802B8151805D700BD8A48B82D5
:100B100000008051815D700BD8A48B9281518019A7
:100B2000D8B40790FCEF0AF0F2940101453FFCEFC6
:100B30000AF0462BFCEF0AF09E900101533FFCEFB8
:100B40000AF0542BFCEF0AF09E9211B821EF08F046
:100B5000040066A1ACEF05F08BB4B6EF05F010AC65
:100B6000B6EF05F08B84109CB7EF05F08B94077CF3
:100B700007ACD2EF05F0C274C2B4CCEF05F0C3CF1E
:100B8000B7F5C4CFB8F50501D890B833B733D890CE
:100B9000B833B733D3EF05F0C3CF55F1C4CF56F117
:100BA000D3EF05F0C28207B440EF06F047C14BF126
:100BB00048C14CF149C14DF14AC14EF15EC162F1EB
:100BC0005FC163F160C164F161C165F196C1B6F1C5
:100BD00097C1B7F198C1B8F199C1B9F19AC1BAF109
:100BE0009BC1BBF19CC1BCF19DC1BDF19EC1BEF1D9
:100BF0009FC1BFF1A0C1C0F1A1C1C1F1A2C1C2F1A9
:100C0000A3C1C3F1A4C1C4F1A5C1C5F1A6C1C6F178
:100C1000A7C1C7F1A8C1C8F1A9C1C9F1AAC1CAF148
:100C2000ABC1CBF1ACC1CCF1ADC1CDF1AEC1CEF118
:100C3000AFC1CFF1B0C1D0F1B1C1D1F1B2C1D2F1E8
:100C4000B3C1D3F1B4C1D4F1B5C1D5F1B7C5B9F5CC
:100C5000B8C5BAF5B9C5BBF5BAC5BCF50101555162
:100C60005B2756515C23E86A5D230E2E40EF06F0A9
:100C70005CC157F15DC158F15B6B5C6B5D6B078EBE
:100C80000201002FFCEF0AF03C0E006F1A50E00B3F
:100C9000E00AE866128818BE02D018B4108E00C1AF
:100CA0000CF101C10DF102C10EF103C10FF104C13C
:100CB00010F105C111F106C112F107C113F108C10C
:100CC00014F109C115F10AC116F10BC117F134C1B4
:100CD00035F105012F51000AD8B41AEF07F00501CC
:100CE0002F51010AD8B4A4EF06F005012F51020AD2
:100CF000D8B4E5EF06F005012F51030AD8B4E5EFAB
:100D000006F005012F51040AD8B4E5EF06F00501FD
:100D10002F51050AD8B4E5EF06F005012F51060A58
:100D2000D8B4E5EF06F005012F51070AD8B4E5EF76
:100D300006F005012F51320AD8B4A2EF06F02F6B4E
:100D40001AEF07F01AEF07F005015767AFEF06F04B
:100D50005867AFEF06F05967AFEF06F05A67B3EF89
:100D600006F01AEF07F05BC500F15CC501F15DC547
:100D700002F15EC503F10101010E046F000E056F63
:100D8000000E066F000E076FFEEC2BF000C15BF546
:100D900001C15CF502C15DF503C15EF50067D8EFE6
:100DA00006F00167D8EF06F00267D8EF06F0036798
:100DB0001AEF07F057C55BF558C55CF559C55DF5E9
:100DC0005AC55EF50F881AEF07F005013067EBEFA3
:100DD00006F01AEF07F00FBE00EF07F010A005EFC6
:100DE00007F001014767FCEF06F04867FCEF06F0EB
:100DF0004967FCEF06F04A6700EF07F005EF07F0E0
:100E000007AE05EF07F017EF07F00501312F1AEFD6
:100E100007F03C0E316F302F1AEF07F00101000E82
:100E2000626FE00E636FA50E646F010E656F0501C2
:100E3000306B0F880501666B37B720EF07F06681CE
:100E40000CC100F10DC101F10EC102F10FC103F19E
:100E500010C104F111C105F112C106F113C107F16E
:100E600014C108F115C109F116C10AF117C10BF13E
:100E700035C134F100C10CF101C10DF102C10EF117
:100E800003C10FF104C110F105C111F106C112F146
:100E900007C113F108C114F109C115F10AC116F116
:100EA0000BC117F134C135F101018A675FEF07F01B
:100EB0008B675FEF07F08C675FEF07F08D6763EF7D
:100EC00007F093EF07F08EC100F18FC101F190C1DF
:100ED00002F191C103F10101010E046F000E056FD3
:100EE000000E066F000E076FFEEC2BF000C18EF1B6
:100EF00001C18FF102C190F103C191F1006788EF48
:100F000007F0016788EF07F0026788EF07F00367D3
:100F100093EF07F08AC18EF18BC18FF18CC190F1F4
:100F20008DC191F10F80D57ED5BE6DD0D6CF47F162
:100F3000D7CF48F145C149F1E86AE8CF4AF119BE77
:100F400002D019A0108C109047C100F148C101F1E6
:100F500049C102F14AC103F101010A0E046F000EFA
:100F6000056F000E066F000E076FFEEC2BF003AF4F
:100F70001080010154A7C9EF07F00F9A0F9C0F9E34
:100F80000101000E5E6F600E5F6F3D0E606F080E18
:100F9000616F010147BFD9EF07F04867D9EF07F04C
:100FA0004967D9EF07F04A67D9EF07F0F288FEEFFB
:100FB00007F0F2985E6B5F6B606B616B966B976B83
:100FC000986B996B9A6B9B6B9C6B9D6B9E6B9F6BED
:100FD000A06BA16BA26BA36BA46BA56BA66BA76B9D
:100FE000A86BA96BAA6BAB6BAC6BAD6BAE6BAF6B4D
:100FF000B06BB16BB26BB36BB46BB56BD76AD66ABF
:101000000101456B466B0CC100F10DC101F10EC130
:1010100002F10FC103F110C104F111C105F112C1B8
:1010200006F113C107F114C108F115C109F116C188
:101030000AF117C10BF135C134F1FCEF0AF0FCEFF6
:101040000AF00201002F65EF0AF0D59ED6CF47F1D6
:10105000D7CF48F145C149F1E86AE8CF4AF1D76AEC
:10106000D66A0101456B466BD58E1A50E00BE00A3B
:10107000E866128818BE02D018B4108E17AE1C8C09
:1010800000C10CF101C10DF102C10EF103C10FF15C
:1010900004C110F105C111F106C112F107C113F12C
:1010A00008C114F109C115F10AC116F10BC117F1FC
:1010B00034C135F10FA0109A11B86AEF08F00101A0
:1010C000620E046F010E056F000E066F000E076FB3
:1010D00073EF08F00101A70E046F020E056F000EFA
:1010E000066F000E076F47C100F148C101F149C109
:1010F00002F14AC103F1FEEC2BF003BF86EF08F0CA
:1011000019BE02D019A0108C11B00F800CC100F1D3
:101110000DC101F10EC102F10FC103F110C104F1C3
:1011200011C105F112C106F113C107F114C108F193
:1011300015C109F116C10AF117C10BF135C134F11E
:1011400002013C0E006F00C10CF101C10DF102C1A2
:101150000EF103C10FF104C110F105C111F106C177
:1011600012F107C113F108C114F109C115F10AC147
:1011700016F10BC117F134C135F105012F51000AE9
:10118000D8B46EEF09F005012F51010AD8B4F8EF79
:1011900008F005012F51020AD8B439EF09F0050112
:1011A0002F51030AD8B439EF09F005012F51040A71
:1011B000D8B439EF09F005012F51050AD8B439EF39
:1011C00009F005012F51060AD8B439EF09F00501DD
:1011D0002F51070AD8B439EF09F005012F51320A0F
:1011E000D8B4F6EF08F02F6B6EEF09F06EEF09F050
:1011F0000501576703EF09F0586703EF09F05967D6
:1012000003EF09F05A6707EF09F06EEF09F05BC5CD
:1012100000F15CC501F15DC502F15EC503F101019C
:10122000010E046F000E056F000E066F000E076FB3
:10123000FEEC2BF000C15BF501C15CF502C15DF570
:1012400003C15EF500672CEF09F001672CEF09F090
:1012500002672CEF09F003676EEF09F057C55BF5E5
:1012600058C55CF559C55DF55AC55EF50F886EEF3A
:1012700009F0050130673FEF09F06EEF09F00FBE8E
:1012800054EF09F010A059EF09F00101476750EF42
:1012900009F0486750EF09F0496750EF09F04A67D5
:1012A00054EF09F059EF09F007AE59EF09F06BEF71
:1012B00009F00501312F6EEF09F03C0E316F302F30
:1012C0006EEF09F00101000E626FE00E636FA50E74
:1012D000646F010E656F0501306B0F880501666B49
:1012E00037B774EF09F066810CC100F10DC101F14F
:1012F0000EC102F10FC103F110C104F111C105F1DA
:1013000012C106F113C107F114C108F115C109F1A9
:1013100016C10AF117C10BF135C134F100C10CF14E
:1013200001C10DF102C10EF103C10FF104C110F1B1
:1013300005C111F106C112F107C113F108C114F181
:1013400009C115F10AC116F10BC117F134C135F10C
:1013500001018A67B3EF09F08B67B3EF09F08C677F
:10136000B3EF09F08D67B7EF09F0E7EF09F08EC131
:1013700000F18FC101F190C102F191C103F10101AE
:10138000010E046F000E056F000E066F000E076F52
:10139000FEEC2BF000C18EF101C18FF102C190F182
:1013A00003C191F10067DCEF09F00167DCEF09F0A0
:1013B0000267DCEF09F00367E7EF09F08AC18EF1FD
:1013C0008BC18FF18CC190F18DC191F10F80109084
:1013D00047C100F148C101F149C102F14AC103F11D
:1013E00001010A0E046F000E056F000E066F000E5D
:1013F000076FFEEC2BF003AF1080010154A70DEF37
:101400000AF00F9A0F9C0F9E0101000E5E6F600E96
:101410005F6F3D0E606F080E616F47C100F148C1FC
:1014200001F149C102F14AC103F10101140E046F37
:10143000050E056F000E066F000E076FFEEC2BF019
:1014400003AF26EF0AF0F2884BEF0AF0F2985E6BDA
:101450005F6B606B616B966B976B986B996B9A6B1C
:101460009B6B9C6B9D6B9E6B9F6BA06BA16BA26B30
:10147000A36BA46BA56BA66BA76BA86BA96BAA6BE0
:10148000AB6BAC6BAD6BAE6BAF6BB06BB16BB26B90
:10149000B36BB46BB56B0CC100F10DC101F10EC1A2
:1014A00002F10FC103F110C104F111C105F112C124
:1014B00006F113C107F114C108F115C109F116C1F4
:1014C0000AF117C10BF135C134F104008BB470EF90
:1014D0000AF010AC70EF0AF08B84109C71EF0AF0E8
:1014E0008B94077C07AC8CEF0AF0C274C2B486EF11
:1014F0000AF0C3CFB7F5C4CFB8F50501D890B8331B
:10150000B733D890B833B7338DEF0AF0C3CF55F166
:10151000C4CF56F18DEF0AF0C28207B4FAEF0AF099
:1015200047C14BF148C14CF149C14DF14AC14EF19F
:101530005EC162F15FC163F160C164F161C165F1D7
:1015400096C1B6F197C1B7F198C1B8F199C1B9F197
:101550009AC1BAF19BC1BBF19CC1BCF19DC1BDF167
:101560009EC1BEF19FC1BFF1A0C1C0F1A1C1C1F137
:10157000A2C1C2F1A3C1C3F1A4C1C4F1A5C1C5F107
:10158000A6C1C6F1A7C1C7F1A8C1C8F1A9C1C9F1D7
:10159000AAC1CAF1ABC1CBF1ACC1CCF1ADC1CDF1A7
:1015A000AEC1CEF1AFC1CFF1B0C1D0F1B1C1D1F177
:1015B000B2C1D2F1B3C1D3F1B4C1D4F1B5C1D5F147
:1015C000B7C5B9F5B8C5BAF5B9C5BBF5BAC5BCF567
:1015D000010155515B2756515C23E86A5D230E2EAD
:1015E000FAEF0AF05CC157F15DC158F15B6B5C6BBF
:1015F0005D6B078EFCEF0AF002C0E0FF005001C0F7
:10160000D8FF1000A6B202EF0BF00CC0A9FF0BC070
:10161000A8FFA69EA69CA684F29E550EA76EAA0EB3
:10162000A76EA682F28EA694A6B214EF0BF00C2A37
:101630001200A96EA69EA69CA680A8500C2A120095
:1016400004012C0E826F6EEC0EF0F9EC2CF00C50B5
:1016500019EC0BF0E8CF00F10C5019EC0BF0E8CFCF
:1016600001F101AF39EF0BF00101FF0E026FFF0E28
:10167000036F9CEC2CF0296745EF0BF00401200E62
:10168000826F6EEC0EF04AEF0BF004012D0E826FAC
:101690006EEC0EF0C6EC2AF01200076A0F6A106AB0
:1016A000116A126A136A0F010D0EC16E860EC06EAA
:1016B000030EC26E0F01680E896E130E926E080E35
:1016C0008A6EF30E936E8B6A900E946EC80E19ECB0
:1016D0000BF0E8CFE8FF1098E8A0108810A805D01C
:1016E0000E0E226E8E0E236E04D00F0E226E8F0E03
:1016F000236E78EC2DF0F18EF19EFC0E19EC0BF0C0
:10170000E8CF0BF00BA011800BA211820BA4118467
:101710000BA81188C90E19EC0BF0E8CF17F0CA0E10
:1017200019EC0BF0E8CF18F0CB0E19EC0BF0E8CF6A
:1017300019F0CC0E19EC0BF0E8CF1AF0CD0E19EC25
:101740000BF0E8CF2FF01C6A1D6A0E6A01015B6B7B
:101750005C6B5D6B576B586BF29A0101476B486B82
:10176000496B4A6B4B6B4C6B4D6B4E6B4F6B506BBD
:10177000516B526B456B466BD76AD66A0F01280EC8
:10178000D56EF28A9D90B00ECD6E01015E6B5F6BDF
:10179000606B616B626B636B646B656B666B676BD5
:1017A000686B696B536B546BCF6ACE6A0F9A0F9C50
:1017B0000F9E9D80760ECA6E9D8202013C0E006FC8
:1017C000CC6A160E19EC0BF0E8CF00F1170E19ECED
:1017D0000BF0E8CF01F1180E19EC0BF0E8CF02F195
:1017E000190E19EC0BF0E8CF03F1010103AF13EF71
:1017F0000CF0F9EC2CF0160E0C6E00C10BF002ECA4
:101800000BF0170E0C6E01C10BF002EC0BF0180E72
:101810000C6E02C10BF002EC0BF0190E0C6E03C142
:101820000BF002EC0BF000C18AF101C18BF102C197
:101830008CF103C18DF100C18EF101C18FF102C1A4
:1018400090F103C191F11A0E19EC0BF0E8CF00F101
:101850001B0E19EC0BF0E8CF01F11C0E19EC0BF08C
:10186000E8CF02F11D0E19EC0BF0E8CF03F10101F6
:1018700003AF69EF0CF0F9EC2CF01A0E0C6E00C1FE
:101880000BF002EC0BF01B0E0C6E01C10BF002EC26
:101890000BF01C0E0C6E02C10BF002EC0BF01D0ED7
:1018A0000C6E03C10BF002EC0BF01A0E19EC0BF0EE
:1018B000E8CF00F11B0E19EC0BF0E8CF01F11C0E84
:1018C00019EC0BF0E8CF02F11D0E19EC0BF0E8CF8C
:1018D00003F100C192F101C193F102C194F103C17E
:1018E00095F1240EAC6E900EAB6E240EAC6E080E0D
:1018F000B86E000EB06E1F0EAF6E0401806B816B70
:101900000F01900EAB6E0F019D8A0301806B816BFE
:10191000C26B8B9200EC32F000EC32F05CEC33F0F6
:10192000DFEC2FF0200E19EC0BF0E8CF2FF50501BE
:101930002F51FF0AD8A4A4EF0CF02F6B200E0C6ED1
:101940002FC50BF002EC0BF00501010E306F3C0EC1
:10195000316F250E19EC0BF0E8CF00F1260E19ECD3
:101960000BF0E8CF01F1270E19EC0BF0E8CF02F1F4
:10197000280E19EC0BF0E8CF03F1010103AFDBEF08
:101980000CF0F9EC2CF0250E0C6E00C10BF002EC03
:101990000BF0260E0C6E01C10BF002EC0BF0270EC3
:1019A0000C6E02C10BF002EC0BF0280E0C6E03C1A2
:1019B0000BF002EC0BF000C157F501C158F502C164
:1019C00059F503C15AF500C15BF501C15CF502C1CF
:1019D0005DF503C15EF5290E19EC0BF0E8CF5FF55C
:1019E000050160515F5DD8A05FC560F505012F510D
:1019F000020A0EE181B808EF0DF00501602F05EF36
:101A00000DF05FC560F508EF0DF081BA9BEF33F084
:101A1000210E19EC0BF0E8CF00F1220E19EC0BF0BF
:101A2000E8CF01F1230E19EC0BF0E8CF02F1240E00
:101A300019EC0BF0E8CF03F1010103AF4EEF0DF00D
:101A4000F9EC2CF0210E0C6E00C10BF002EC0BF047
:101A5000220E0C6E01C10BF002EC0BF0230E0C6E8B
:101A600002C10BF002EC0BF0240E0C6E03C10BF064
:101A700002EC0BF0210E19EC0BF0E8CF00F1220E76
:101A800019EC0BF0E8CF01F1230E19EC0BF0E8CFC5
:101A900002F1240E19EC0BF0E8CF03F100C161F55F
:101AA00001C162F502C163F503C164F527EC2FF0B3
:101AB00029EC2EF081EC2DF005012F51030A12E0E4
:101AC00005012F51040A1DE005012F51050A24E0EC
:101AD00005012F51060A32E005012F51070A38E0AF
:101AE000B1EF0DF0B0C500F101010F0E00170101BB
:101AF0000051000A36E001010051050A32E0AEEF64
:101B00000DF0B0C500F101010F0E001701010051E9
:101B1000000A27E0AEEF0DF00501B051000A21E008
:101B20000501B051150A1DE00501B051300A19E058
:101B30000501B051450A15E0AEEF0DF00501B051B9
:101B4000000A0FE00501B051300A0BE0AEEF0DF0D6
:101B50000501B051000A05E0AEEF0DF081BA9BEF30
:101B600033F007900001F28EF28C12AE03D012BC5B
:101B7000ADEF18F007B048EF29F00FB0E4EF22F016
:101B800010BEE4EF22F012B8E4EF22F00FB881EFBC
:101B90001CF00301805181197F0BD8B448EF29F064
:101BA00013EE00F081517F0BE126812BE7CFE8FF98
:101BB000E00BD8B448EF29F023EE82F0C2513F0B7E
:101BC000D926E7CFDFFFC22BDF50780AD8A448EF31
:101BD00029F007808EC100F18FC101F190C102F19F
:101BE00091C103F10101040E046F000E056F000E98
:101BF000066F000E076FFEEC2BF000AF09EF0EF042
:101C00000101030E8E6F000E8F6F000E906F000E9D
:101C1000916F03018251720AD8B4C9EF22F0825148
:101C2000520AD8B4C9EF22F08251750AD8B4C9EF6C
:101C300022F08251630AD8B402EF26F08251690A79
:101C4000D8B478EF1FF082517A0AD8B48BEF20F025
:101C50008251490AD8B417EF1FF08251500AD8B404
:101C600035EF1EF08251700AD8B478EF1EF0825121
:101C7000540AD8B4A3EF1EF08251740AD8B4E9EF25
:101C80001EF08251410AD8B484EF0FF082514B0A02
:101C9000D8B482EF0EF082516D0AD8B4B7EF13F0CA
:101CA00082514D0AD8B4D0EF13F08251730AD8B4E0
:101CB000F9EF21F08251530AD8B45EEF22F082513D
:101CC0004C0AD8B45FEF14F08251590AD8B408EF27
:101CD00013F012AE01D0128C39EF26F0040114EE8D
:101CE00000F080517F0BE12682C4E7FF802B1200B9
:101CF00004010D0E826F6EEC0EF00A0E826F6EEC18
:101D00000EF0120004014B0E826F6EEC0EF0040117
:101D10002C0E826F6EEC0EF081B802D02FB630D050
:101D200003018351430AD8B4C7EF0EF00301835176
:101D3000630AD8B4C9EF0EF003018351520AD8B434
:101D4000CBEF0EF003018351720AD8B4CDEF0EF041
:101D500003018351470AD8B4CFEF0EF0030183513A
:101D6000670AD8B4D1EF0EF003018351540AD8B4F6
:101D7000D3EF0EF003018351740AD8B442EF0FF091
:101D800003018351550AD8B4D5EF0EF082D02F80CD
:101D90007AD02F9078D02F8276D02F9274D02F8443
:101DA00072D02F9470D02F866ED084C330F185C34B
:101DB00031F186C332F187C333F10101296B47EC5E
:101DC0002DF0BEEC2CF000C104F101C105F102C1FF
:101DD00006F103C107F13AEC2DF0200EF86EF76A18
:101DE000F66A0900F5CF2CF10900F5CF2DF10900B5
:101DF000F5CF2EF10900F5CF2FF10900F5CF30F125
:101E00000900F5CF31F10900F5CF32F10900F5CF26
:101E100033F10101296B47EC2DF0BEEC2CF0FEEC08
:101E20002BF000671BEF0FF001671BEF0FF002674D
:101E30001BEF0FF0036701D025D004014E0E826F17
:101E40006EEC0EF004016F0E826F6EEC0EF004016A
:101E50004D0E826F6EEC0EF00401610E826F6EEC1F
:101E60000EF00401740E826F6EEC0EF00401630E2E
:101E7000826F6EEC0EF00401680E826F6EEC0EF055
:101E800037EF26F02F96CD0E0C6E2FC00BF002EC24
:101E90000BF0CD0E19EC0BF0E8CF2FF02FB006D0E1
:101EA0000401630E826F6EEC0EF005D00401430E48
:101EB000826F6EEC0EF02FB206D00401720E826FAC
:101EC0006EEC0EF005D00401520E826F6EEC0EF037
:101ED0002FB406D00401670E826F6EEC0EF005D0B1
:101EE0000401470E826F6EEC0EF02FB606D004018F
:101EF000740E826F6EEC0EF005D00401540E826FEA
:101F00006EEC0EF037EF26F00401410E826F6EEC9E
:101F10000EF003018351310AD8B428EF12F0030107
:101F20008351320AD8B458EF11F003018351330AB8
:101F3000D8B4E1EF10F003018351340AD8B4D1EFE3
:101F40000FF003018351350AD8B4AEEF0FF004014E
:101F50003F0E826F6EEC0EF037EF26F004012C0E70
:101F6000826F6EEC0EF003018451300AD8B4C1EFD9
:101F70000FF003018451310AD8B4C9EF0FF01AEF02
:101F800011F08B900401300E826F6EEC0EF0CFEFEB
:101F90000FF08B800401310E826F6EEC0EF037EF84
:101FA00026F0CC0E19EC0BF0E8CF0BF004012C0E50
:101FB000826F6EEC0EF003018451310AD8B4F5EF54
:101FC0000FF003018451300AD8B4F7EF0FF003018A
:101FD00084514D0AD8B401EF10F003018451540A22
:101FE000D8B408EF10F01FEF10F08A8401D08A9463
:101FF0000BAE04D00BAC02D00BBA21D0E00E0B120A
:1020000018D01F0E0B168539E844E00B0B1211D0C7
:10201000E00E0B163AEC2DF085C332F186C333F196
:102020000101296B47EC2DF0BEEC2CF000511F0B89
:102030000B12CC0E0C6E0BC00BF002EC0BF004017B
:10204000340E826F6EEC0EF004012C0E826F6EEC7B
:102050000EF0CC0E19EC0BF0E8CF1AF08AB406D0D3
:102060000401300E826F6EEC0EF005D00401310ECB
:10207000826F6EEC0EF004012C0E826F6EEC0EF08F
:102080001A38E840070BE8CF82F40401300E8227AB
:102090006EEC0EF004012C0E826F6EEC0EF0F9EC7B
:1020A0002CF01A501F0BE8CF00F19CEC2CF032C141
:1020B00082F40401300E82276EEC0EF033C182F4FC
:1020C0000401300E82276EEC0EF004012C0E826F9C
:1020D0006EEC0EF0F9EC2CF02DC000F100AF0BD03F
:1020E000FF0E016FFF0E026FFF0E036F04012D0E36
:1020F000826F6EEC0EF09CEC2CF031C182F4040186
:10210000300E82276EEC0EF032C182F40401300EE4
:1021100082276EEC0EF033C182F40401300E822768
:102120006EEC0EF004012C0E826F6EEC0EF0F9ECEA
:102130002CF02CC000F19CEC2CF031C182F4040195
:10214000300E82276EEC0EF032C182F40401300EA4
:1021500082276EEC0EF033C182F40401300E822728
:102160006EEC0EF004012C0E826F6EEC0EF0F9ECAA
:102170002CF02EC000F100AF0BD0FF0E016FFF0E50
:10218000026FFF0E036F04012D0E826F6EEC0EF0D6
:102190009CEC2CF031C182F40401300E82276EECED
:1021A0000EF032C182F40401300E82276EEC0EF084
:1021B00033C182F40401300E82276EEC0EF037EF4B
:1021C00026F0CB0E19EC0BF0E8CF0BF004012C0E2F
:1021D000826F6EEC0EF003018451450AD8B405EF0E
:1021E00011F003018451440AD8B408EF11F003013F
:1021F0008451300AD8B40BEF11F003018451310A35
:10220000D8B40FEF11F01AEF11F00B9E14EF11F08C
:102210000B8E14EF11F0FC0E0B1614EF11F0FC0EE8
:102220000B160B8014EF11F0CB0E0C6E0BC00BF0E5
:1022300002EC0BF00401330E826F6EEC0EF0040121
:102240002C0E826F6EEC0EF0CB0E19EC0BF0E8CF7B
:1022500019F019BE33EF11F00401450E826F6EECD8
:102260000EF038EF11F00401440E826F6EEC0EF0A8
:1022700004012C0E826F6EEC0EF00401300E826FA2
:102280006EEC0EF004012C0E826F6EEC0EF019B0A5
:1022900051EF11F00401300E826F6EEC0EF056EF2C
:1022A00011F00401310E826F6EEC0EF037EF26F064
:1022B000CA0E19EC0BF0E8CF0BF004012C0E826F64
:1022C0006EEC0EF003018451450AD8B494EF11F07E
:1022D00003018451440AD8B497EF11F003018451EB
:1022E0004D0AD8B4A0EF11F003018451410AD8B4CB
:1022F0009AEF11F003018451460AD8B49DEF11F012
:1023000003018451560AD8B4A8EF11F00301845197
:10231000500AD8B4B3EF11F003018451520AD8B473
:10232000B6EF11F0BFEF11F00B9EB9EF11F00B8E6D
:10233000B9EF11F00B9CB9EF11F00B8CB9EF11F064
:10234000FC0E0B1685C3E8FF030B0B12B9EF11F05F
:10235000C70E0B1685C3E8FF070BE846E846E846BC
:102360000B12B9EF11F00B84B9EF11F00B94B9EF28
:1023700011F0CA0E0C6E0BC00BF002EC0BF0CA0E83
:1023800019EC0BF0E8CF18F00401320E826F6EECFE
:102390000EF004012C0E826F6EEC0EF018BED8EF1A
:1023A00011F00401450E826F6EEC0EF0DDEF11F0BE
:1023B0000401440E826F6EEC0EF004012C0E826F4D
:1023C0006EEC0EF018C0E8FF030BE8CF82F40401B6
:1023D000300E82276EEC0EF004012C0E826F6EEC34
:1023E0000EF018BCFBEF11F00401410E826F6EEC91
:1023F0000EF000EF12F00401460E826F6EEC0EF04C
:1024000004012C0E826F6EEC0EF018C0E8FF380B42
:10241000E842E842E842E8CF82F40401300E822725
:102420006EEC0EF004012C0E826F6EEC0EF018B400
:1024300021EF12F00401520E826F6EEC0EF026EFC7
:1024400012F00401500E826F6EEC0EF037EF26F0A2
:10245000C90E19EC0BF0E8CF0BF004012C0E826FC3
:102460006EEC0EF003018451450AD8B446EF12F029
:1024700003018451440AD8B449EF12F00301845196
:102480004D0AD8B44CEF12F05AEF12F00B9E54EFF5
:1024900012F00B8E54EF12F0F80E0B1685C3E8FF06
:1024A000070B0B1254EF12F0C90E0C6E0BC00BF0A1
:1024B00002EC0BF00401310E826F6EEC0EF00401A1
:1024C0002C0E826F6EEC0EF0C90E19EC0BF0E8CFFB
:1024D00017F017BE06D00401450E826F6EEC0EF0A9
:1024E00005D00401440E826F6EEC0EF004012C0E38
:1024F000826F6EEC0EF017C0E8FF070BE8CF82F496
:102500000401300E82276EEC0EF004012C0E826F57
:102510006EEC0EF00780F9EC2CF028C0E8FF003BD1
:1025200000430043030B9CEC2CF033C182F4040104
:10253000300E82276EEC0EF004012C0E826F6EECD2
:102540000EF0F9EC2CF028C001F1019F019D29C08B
:1025500000F101019CEC2CF02FC182F40401300E3B
:1025600082276EEC0EF030C182F40401300E822717
:102570006EEC0EF031C182F40401300E82276EEC55
:102580000EF032C182F40401300E82276EEC0EF0A0
:1025900033C182F40401300E82276EEC0EF0040188
:1025A0002C0E826F6EEC0EF0F9EC2CF02AC001F1CB
:1025B0002BC000F1D89001330033D89001330033A1
:1025C00001019CEC2CF02FC182F40401300E822713
:1025D0006EEC0EF030C182F40401300E82276EECF6
:1025E0000EF031C182F40401300E82276EEC0EF041
:1025F00032C182F40401300E82276EEC0EF033C13A
:1026000082F40401300E82276EEC0EF037EF26F0D4
:10261000FC0E19EC0BF0E8CF0BF003018351520ACA
:10262000D8B43FEF13F003018351720AD8B442EFDC
:1026300013F003018351500AD8B445EF13F003019E
:102640008351700AD8B448EF13F003018351550A3F
:10265000D8B44BEF13F003018351750AD8B44EEF91
:1026600013F003018351430AD8B457EF13F0030169
:102670008351630AD8B45AEF13F063EF13F00B9051
:102680005DEF13F00B805DEF13F00B925DEF13F035
:102690000B825DEF13F00B945DEF13F00B845DEF95
:1026A00013F00B965DEF13F00B865DEF13F00B98B4
:1026B0005DEF13F00B885DEF13F0FC0E0C6E0BC09A
:1026C0000BF002EC0BF00401590E826F6EEC0EF071
:1026D0001190119211941198FC0E19EC0BF0E8CFA7
:1026E0000BF00BA011800BA211820BA411840BA87C
:1026F000118811A083EF13F00401520E826F6EEC6B
:102700000EF088EF13F00401720E826F6EEC0EF083
:1027100011A892EF13F00401430E826F6EEC0EF0DD
:1027200097EF13F00401630E826F6EEC0EF011A2AE
:10273000A1EF13F00401500E826F6EEC0EF0A6EFC5
:1027400013F00401700E826F6EEC0EF011A4B0EF66
:1027500013F00401550E826F6EEC0EF0B5EF13F01E
:102760000401750E826F6EEC0EF037EF26F0040157
:102770006D0E826F6EEC0EF003018351300AD8B4F7
:102780000FEF14F003018351310AD8B422EF14F093
:1027900003018351320AD8B435EF14F039EF26F033
:1027A00004014D0E826F6EEC0EF03AEC2DF084C3F6
:1027B00031F185C332F186C333F10101296B47EC56
:1027C0002DF0BEEC2CF003018351300AD8B4F7EFA2
:1027D00013F003018351310AD8B4FFEF13F0030162
:1027E0008351320AD8B407EF14F039EF26F0FD0E0A
:1027F0000C6E00C10BF002EC0BF00FEF14F0FE0EAC
:102800000C6E00C10BF002EC0BF022EF14F0FF0E87
:102810000C6E00C10BF002EC0BF035EF14F004016C
:10282000300E826F6EEC0EF004012C0E826F6EEC97
:102830000EF0F9EC2CF0FD0E19EC0BF0E8CF00F1E6
:1028400046EF14F00401310E826F6EEC0EF00401BD
:102850002C0E826F6EEC0EF0F9EC2CF0FE0E19ECE3
:102860000BF0E8CF00F146EF14F00401320E826F56
:102870006EEC0EF0F9EC2CF004012C0E826F6EEC75
:102880000EF0FF0E19EC0BF0E8CF00F19CEC2CF0F1
:1028900031C182F40401300E82276EEC0EF032C199
:1028A00082F40401300E82276EEC0EF033C182F404
:1028B0000401300E82276EEC0EF037EF26F0030194
:1028C0008351300AD8B45AEF19F003018351310A09
:1028D000D8B487EF1AF003018351320AD8B4F5EF68
:1028E0001AF003018351330AD8B405EF1BF003013A
:1028F0008351340AD8B415EF1BF003018351350A14
:10290000D8B486EF1CF003018351360AD8B4B4EF73
:102910001CF003018351370AD8B432EF17F00301DA
:102920008351380AD8B4D0EF17F003018351460A17
:10293000D8B4DAEF1BF0030183514D0AD8B4ABEFE2
:1029400015F0030183516D0AD8B4C5EF15F00301EA
:1029500083515A0AD8B401EF1AF003018351490A8E
:10296000D8B4B4EF1DF003018351500AD8B4E6EF98
:102970001CF003018351540AD8B45FEF1DF003012A
:102980008351630AD8B4E5EF15F003018351430A7C
:10299000D8B4DDEF16F003018351730AD8B4E3EF26
:1029A00015F003018351610AD8B4F8EF14F0030164
:1029B0008351650AD8B4AAEF19F003018351450A7F
:1029C000D8B4B8EF19F003018351620AD8B4C6EF46
:1029D00019F003018351420AD8B4D4EF19F003016E
:1029E0008351760AD8B4E2EF19F0D8A439EF26F073
:1029F00004014C0E826F6EEC0EF00401610E826FCA
:102A00006EEC0EF029EC2EF004012C0E826F6EECB1
:102A10000EF0F9EC2CF0AFC500F101019CEC2CF0AC
:102A200031C182F40401300E82276EEC0EF032C107
:102A300082F40401300E82276EEC0EF033C182F472
:102A40000401300E82276EEC0EF004012C0E826F12
:102A50006EEC0EF0F9EC2CF0B0C500F101019CEC2D
:102A60002CF031C182F40401300E82276EEC0EF09E
:102A700032C182F40401300E82276EEC0EF033C1B5
:102A800082F40401300E82276EEC0EF004012C0E4D
:102A9000826F6EEC0EF0F9EC2CF0B1C500F1010183
:102AA0009CEC2CF031C182F40401300E82276EECD4
:102AB0000EF032C182F40401300E82276EEC0EF06B
:102AC00033C182F40401300E82276EEC0EF0040153
:102AD0002C0E826F6EEC0EF0F9EC2CF0B2C500F10A
:102AE00001019CEC2CF031C182F40401300E8227EC
:102AF0006EEC0EF032C182F40401300E82276EECCF
:102B00000EF033C182F40401300E82276EEC0EF019
:102B100004012C0E826F6EEC0EF0F9EC2CF0B6C5B1
:102B200000F101019CEC2CF031C182F40401300E63
:102B300082276EEC0EF032C182F40401300E82273F
:102B40006EEC0EF033C182F40401300E82276EEC7D
:102B50000EF0E2EF1CF03AEC2DF084C333F147ECB9
:102B60002DF0BEEC2CF0200E0C6E00C10BF002EC30
:102B70000BF000C12FF505012F51000A06E00501F9
:102B80002F51010A02E0C3EC2EF004014C0E826FBB
:102B90006EEC0EF004014D0E826F6EEC0EF004012F
:102BA0002C0E826F6EEC0EF0F9EC2CF02FC500F1BC
:102BB0009CEC2CF033C182F40401300E82276EECC1
:102BC0000EF0E2EF1CF09BEF33F004014C0E826F2D
:102BD0006EEC0EF00401630E826F6EEC0EF081EC71
:102BE0002DF004012C0E826F6EEC0EF0FAEC15F055
:102BF000E2EF1CF0F9EC2CF0B5C500F10101003B4F
:102C00000F0E00179CEC2CF033C182F40401300E3F
:102C100082276EEC0EF0B5C500F101010F0E010127
:102C200000179CEC2CF033C182F40401300E822793
:102C30006EEC0EF004012D0E826F6EEC0EF0B4C53A
:102C400000F10101003B0F0E00179CEC2CF033C18A
:102C500082F40401300E82276EEC0EF0B4C500F150
:102C600001010F0E010100179CEC2CF033C182F41E
:102C70000401300E82276EEC0EF004012D0E826FDF
:102C80006EEC0EF0B3C500F10101003B0F0E001712
:102C90009CEC2CF033C182F40401300E82276EECE0
:102CA0000EF0B3C500F101010F0E010100179CECFD
:102CB0002CF033C182F40401300E82276EEC0EF04A
:102CC0000401200E826F6EEC0EF0B2C500F10F0E03
:102CD000010100179CEC2CF033C182F40401300E8A
:102CE00082276EEC0EF00401200E826F6EEC0EF067
:102CF000B1C500F101010101003B0F0E00179CEC72
:102D00002CF033C182F40401300E82276EEC0EF0F9
:102D1000B1C500F101010F0E010100179CEC2CF070
:102D200033C182F40401300E82276EEC0EF00401F0
:102D30003A0E826F6EEC0EF0B0C500F10101003B5F
:102D40000F0E00179CEC2CF033C182F40401300EFE
:102D500082276EEC0EF0B0C500F101010F0E0101EB
:102D600000179CEC2CF033C182F40401300E822752
:102D70006EEC0EF004013A0E826F6EEC0EF0AFC5F1
:102D800000F10101003B0F0E00179CEC2CF033C149
:102D900082F40401300E82276EEC0EF0AFC500F114
:102DA00001010F0E00179CEC2CF033C182F40401DA
:102DB000300E82276EEC0EF0120084C3E8FF0F0B7A
:102DC000E83AE8CFB5F585C3E8FF0F0B0501B51369
:102DD00087C3E8FF0F0BE83AE8CFB4F588C3E8FFF4
:102DE0000F0B0501B4138AC3E8FF0F0BE83AE8CFD5
:102DF000B3F58BC3E8FF0F0B0501B3138DC3E8FFD9
:102E00000F0BE8CFB2F58FC3E8FF0F0BE83AE8CF1E
:102E1000B1F590C3E8FF0F0B0501B11392C3E8FFB2
:102E20000F0BE83AE8CFB0F593C3E8FF0F0B0501AD
:102E3000B01395C3E8FF0F0BE83AE8CFAFF596C3A0
:102E4000E8FF0F0B0501AF13DCEC2DF004014C0E75
:102E5000826F6EEC0EF00401430E826F6EEC0EF08A
:102E6000EFEF15F0078404014C0E826F6EEC0EF04C
:102E70000401370E826F6EEC0EF004012C0E826F8F
:102E80006EEC0EF005012E51130A06E005012E51DD
:102E9000170A0DE0CDEF17F00101000E006F000ED4
:102EA000016F100E026F000E036F60EF17F001014B
:102EB000000E006F000E016F000E026F010E036F17
:102EC0009CEC2CF02AC182F40401300E82276EECB7
:102ED0000EF02BC182F40401300E82276EEC0EF04E
:102EE0002CC182F40401300E82276EEC0EF02DC14D
:102EF00082F40401300E82276EEC0EF02EC182F4B3
:102F00000401300E82276EEC0EF02FC182F4040112
:102F1000300E82276EEC0EF030C182F40401300EC8
:102F200082276EEC0EF031C182F40401300E82274C
:102F30006EEC0EF032C182F40401300E82276EEC8A
:102F40000EF033C182F40401300E82276EEC0EF0D5
:102F500004012C0E826F6EEC0EF00101100E006F5A
:102F6000000E016F000E026F000E036F9CEC2CF040
:102F700031C182F40401300E82276EEC0EF032C1B2
:102F800082F40401300E82276EEC0EF033C182F41D
:102F90000401300E82276EEC0EF00794E2EF1CF075
:102FA0000501216B226B236B246B04014C0E826F95
:102FB0006EEC0EF00401380E826F6EEC0EF0040120
:102FC0002C0E826F6EEC0EF00101100E006F000EE1
:102FD000016F000E026F000E036F9CEC2CF02AC1F3
:102FE00082F40401300E82276EEC0EF02BC182F4C5
:102FF0000401300E82276EEC0EF02CC182F4040125
:10300000300E82276EEC0EF02DC182F40401300EDA
:1030100082276EEC0EF02EC182F40401300E82275E
:103020006EEC0EF02FC182F40401300E82276EEC9C
:103030000EF030C182F40401300E82276EEC0EF0E7
:1030400031C182F40401300E82276EEC0EF032C1E1
:1030500082F40401300E82276EEC0EF033C182F44C
:103060000401300E82276EEC0EF004012C0E826FEC
:103070006EEC0EF025C500F126C501F127C502F161
:1030800028C503F10101100E046F000E056F000E3C
:10309000066F000E076F2FEC2CF000C133F501C155
:1030A00034F502C135F503C136F59CEC2CF02AC18C
:1030B00082F40401300E82276EEC0EF02BC182F4F4
:1030C0000401300E82276EEC0EF02CC182F4040154
:1030D000300E82276EEC0EF02DC182F40401300E0A
:1030E00082276EEC0EF02EC182F40401300E82278E
:1030F0006EEC0EF02FC182F40401300E82276EECCC
:103100000EF030C182F40401300E82276EEC0EF016
:1031100031C182F40401300E82276EEC0EF032C110
:1031200082F40401300E82276EEC0EF033C182F47B
:103130000401300E82276EEC0EF078EC0EF00501E3
:103140003367AAEF18F03467AAEF18F03567AAEFD3
:1031500018F0366702D049EF19F0129E129C21C573
:1031600000F122C501F123C502F124C503F1899ABA
:10317000400EC76E200EC66E9E96C69E0B0EC96E82
:10318000FF0E9EB602D0E82EFCD79E96C69E02C1C8
:10319000C9FFFF0E9EB602D0E82EFCD79E96C69EB3
:1031A00001C1C9FFFF0E9EB602D0E82EFCD79E9645
:1031B000C69E00C1C9FFFF0E9EB602D0E82EFCD706
:1031C0009E96C69EC952FF0E9EB602D0E82EFCD730
:1031D0000501100E326F040114EE00F080517F0BD8
:1031E000E1269E96C69EC952FF0E9EB602D0E82EDC
:1031F000FCD7C9CFE7FF0401802B0501322FEBEF8D
:1032000018F0898A33C500F134C501F135C502F1E2
:1032100036C503F10101010E046F000E056F000EAB
:10322000066F000E076FFEEC2BF000C133F501C1F5
:1032300034F502C135F503C136F50501336728EFD2
:1032400019F0346728EF19F0356728EF19F0366761
:1032500002D049EF19F021C500F122C501F123C5C3
:1032600002F124C503F10101100E046F000E056F79
:10327000000E066F000E076F03EC2CF000C121F565
:1032800001C122F502C123F503C124F5128E39EFE5
:1032900026F00401450E826F6EEC0EF004014F0E15
:1032A000826F6EEC0EF00401460E826F6EEC0EF033
:1032B000E2EF1CF007845CEC33F0F9EC2CF02DC548
:1032C00000F19CEC2CF004014C0E826F6EEC0EF0C1
:1032D0000401300E826F6EEC0EF004012C0E826F32
:1032E0006EEC0EF031C182F40401300E82276EECD8
:1032F0000EF032C182F40401300E82276EEC0EF023
:1033000033C182F40401300E82276EEC0EF004010A
:103310002C0E826F6EEC0EF0F9EC2CF02EC500F145
:103320009CEC2CF031C182F40401300E82276EEC4B
:103330000EF032C182F40401300E82276EEC0EF0E2
:1033400033C182F40401300E82276EEC0EF0079434
:10335000E2EF1CF004014C0E826F6EEC0EF00401E3
:10336000650E826F6EEC0EF083EC2FF0E2EF1CF036
:1033700004014C0E826F6EEC0EF00401450E826F5C
:103380006EEC0EF09AEC2FF0E2EF1CF004014C0E04
:10339000826F6EEC0EF00401620E826F6EEC0EF026
:1033A000C8EC2FF0E2EF1CF004014C0E826F6EECC3
:1033B0000EF00401420E826F6EEC0EF0B1EC2FF0B5
:1033C000E2EF1CF004014C0E826F6EEC0EF0040173
:1033D000760E826F6EEC0EF004012C0E826F6EEC96
:1033E0000EF010A807D00401310E826F6EEC0EF0C3
:1033F000E2EF1CF00401300E826F6EEC0EF0E2EF93
:103400001CF004014C0E826F6EEC0EF004015A0E9B
:10341000826F6EEC0EF004012C0E826F6EEC0EF0DB
:103420005CEC33F0F9EC2CF005012E51130A06E0A8
:1034300005012E51170A0DE032EF1AF00101000EBE
:10344000006F000E016F100E026F000E036F32EF5F
:103450001AF00101000E006F000E016F000E026FE6
:10346000010E036F0101100E046F000E056F000EB8
:10347000066F000E076F2FEC2CF09CEC2CF02AC18D
:1034800082F40401300E82276EEC0EF02BC182F420
:103490000401300E82276EEC0EF02CC182F4040180
:1034A000300E82276EEC0EF02DC182F40401300E36
:1034B00082276EEC0EF02EC182F40401300E8227BA
:1034C0006EEC0EF02FC182F40401300E82276EECF8
:1034D0000EF030C182F40401300E82276EEC0EF043
:1034E00031C182F40401300E82276EEC0EF032C13D
:1034F00082F40401300E82276EEC0EF033C182F4A8
:103500000401300E82276EEC0EF0E2EF1CF007840F
:1035100004014C0E826F6EEC0EF00401310E826FCE
:103520006EEC0EF004012C0E826F6EEC0EF025C5D1
:1035300000F126C501F127C502F128C503F10101FB
:10354000100E046F000E056F000E066F000E076F61
:103550002FEC2CF09CEC2CF02AC182F40401300EEC
:1035600082276EEC0EF02BC182F40401300E82270C
:103570006EEC0EF02CC182F40401300E82276EEC4A
:103580000EF02DC182F40401300E82276EEC0EF095
:103590002EC182F40401300E82276EEC0EF02FC192
:1035A00082F40401300E82276EEC0EF030C182F4FA
:1035B0000401300E82276EEC0EF031C182F404015A
:1035C000300E82276EEC0EF032C182F40401300E10
:1035D00082276EEC0EF033C182F40401300E822794
:1035E0006EEC0EF00794E2EF1CF0078404014C0E21
:1035F000826F6EEC0EF00401320E826F6EEC0EF0F4
:10360000B6EC31F00794E2EF1CF0078404014C0E95
:10361000826F6EEC0EF00401330E826F6EEC0EF0D2
:1036200013EC32F0079492EF1AF0078404014C0E69
:10363000826F6EEC0EF00401340E826F6EEC0EF0B1
:1036400004012C0E826F6EEC0EF03AEC2DF084C368
:103650002AF185C32BF186C32CF187C32DF188C3D2
:103660002EF189C32FF18AC330F18BC331F18CC3A2
:1036700032F18DC333F10101296B47EC2DF0BEEC23
:103680002CF0100E046F000E056F000E066F000E7A
:10369000076F0FEC2CF000C121F501C122F502C12A
:1036A00023F503C124F50FEC33F038C5AFF539C568
:1036B000B0F53AC5B1F53BC5B2F53CC5B3F53DC56E
:1036C000B4F53EC5B5F5FAEC15F004012C0E826F89
:1036D0006EEC0EF03FC500F140C501F141C502F1AD
:1036E00042C503F10101000E046F000E056F010ECB
:1036F000066F000E076F2FEC2CF09CEC2CF0296766
:1037000084EF1BF089EF1BF004012D0E826F6EEC2D
:103710000EF030C182F40401300E82276EEC0EF000
:1037200031C182F40401300E82276EEC0EF00401E8
:103730002E0E826F6EEC0EF032C182F40401300E58
:1037400082276EEC0EF033C182F40401300E822722
:103750006EEC0EF004012C0E826F6EEC0EF0F9ECA4
:103760002CF043C500F144C501F163EC27F00401DE
:103770002C0E826F6EEC0EF0F9EC2CF045C500F1CA
:103780009CEC2CF031C182F40401300E82276EECE7
:103790000EF032C182F40401300E82276EEC0EF07E
:1037A00033C182F40401300E82276EEC0EF00794D0
:1037B000E2EF1CF03AEC2DF085C32AF186C32BF121
:1037C00087C32CF188C32DF189C32EF18AC32FF151
:1037D0008BC330F18CC331F18DC332F18EC333F121
:1037E0000101296B47EC2DF0BEEC2CF00101010E1C
:1037F000046F000E056F000E066F000E076FFEECE3
:103800002BF0100E046F000E056F000E066F000EF9
:10381000076F0FEC2CF000C129F501C12AF502C198
:103820002BF503C12CF53DEC31F004014C0E826FF9
:103830006EEC0EF00401460E826F6EEC0EF0040189
:103840002C0E826F6EEC0EF025C500F126C501F13D
:1038500027C502F128C503F10101100E046F000E07
:10386000056F000E066F000E076F2FEC2CF09CEC1E
:103870002CF02AC182F40401300E82276EEC0EF087
:103880002BC182F40401300E82276EEC0EF02CC1A5
:1038900082F40401300E82276EEC0EF02DC182F40A
:1038A0000401300E82276EEC0EF02EC182F404016A
:1038B000300E82276EEC0EF02FC182F40401300E20
:1038C00082276EEC0EF030C182F40401300E8227A4
:1038D0006EEC0EF031C182F40401300E82276EECE2
:1038E0000EF032C182F40401300E82276EEC0EF02D
:1038F00033C182F40401300E82276EEC0EF0E2EF49
:103900001CF00F9813EC32F039EF26F004014C0E46
:10391000826F6EEC0EF00401350E826F6EEC0EF0CD
:1039200004012C0E826F6EEC0EF0F9EC2CF0078483
:10393000B9C500F107949CEC2CF031C182F404016C
:10394000300E82276EEC0EF032C182F40401300E8C
:1039500082276EEC0EF033C182F40401300E822710
:103960006EEC0EF0E2EF1CF0D6EC31F0F9EC2CF03E
:1039700037C500F19CEC2CF004014C0E826F6EEC0C
:103980000EF00401360E826F6EEC0EF004012C0E68
:10399000826F6EEC0EF031C182F40401300E82278A
:1039A0006EEC0EF032C182F40401300E82276EEC10
:1039B0000EF033C182F40401300E82276EEC0EF05B
:1039C000E2EF1CF078EC0EF039EF26F004014C0E1B
:1039D000826F6EEC0EF00401500E826F6EEC0EF0F2
:1039E00004012C0E826F6EEC0EF085C32AF186C3A3
:1039F0002BF187C32CF188C32DF189C32EF18AC323
:103A00002FF18BC330F18CC331F18DC332F18EC3F2
:103A100033F1010147EC2DF0BEEC2CF00301845191
:103A2000530A0DE0030184514D0A38E00401780E79
:103A3000826F6EEC0EF078EC0EF039EF26F0040198
:103A4000530E826F6EEC0EF0250E0C6E00C10BF063
:103A500002EC0BF0260E0C6E01C10BF002EC0BF029
:103A6000270E0C6E02C10BF002EC0BF0280E0C6E50
:103A700003C10BF002EC0BF000C157F501C158F582
:103A800002C159F503C15AF500C15BF501C15CF5EE
:103A900002C15DF503C15EF5C3EF1DF004014D0EDB
:103AA000826F6EEC0EF0290E0C6E00C10BF002EC72
:103AB0000BF000C15FF500C160F5C3EF1DF004011C
:103AC0004C0E826F6EEC0EF00401540E826F6EECA1
:103AD0000EF004012C0E826F6EEC0EF084C32AF1FE
:103AE00085C32BF186C32CF187C32DF188C32EF13A
:103AF00089C32FF18AC330F18BC331F18DC332F109
:103B00008EC333F1010147EC2DF0BEEC2CF0010126
:103B1000000E046F000E056F010E066F000E076F9A
:103B20000FEC2CF0210E0C6E00C10BF002EC0BF030
:103B3000220E0C6E01C10BF002EC0BF0230E0C6E8A
:103B400002C10BF002EC0BF0240E0C6E03C10BF063
:103B500002EC0BF000C161F501C162F502C163F531
:103B600003C164F5C3EF1DF004014C0E826F6EECCF
:103B70000EF00401490E826F6EEC0EF004012C0E63
:103B8000826F6EEC0EF0250E19EC0BF0E8CF00F111
:103B9000260E19EC0BF0E8CF01F1270E19EC0BF013
:103BA000E8CF02F1280E19EC0BF0E8CF03F19CEC02
:103BB0002CF07FEC2AF00401730E826F6EEC0EF095
:103BC00004012C0E826F6EEC0EF0F9EC2CF0290E35
:103BD00019EC0BF0E8CF00F19CEC2CF07FEC2AF014
:103BE0000401730E826F6EEC0EF004012C0E826FD6
:103BF0006EEC0EF05BC500F15CC501F15DC502F134
:103C00005EC503F19CEC2CF07FEC2AF00401730EEE
:103C1000826F6EEC0EF004012C0E826F6EEC0EF0D3
:103C2000F9EC2CF060C500F19CEC2CF07FEC2AF054
:103C300004016D0E826F6EEC0EF004012C0E826F8B
:103C40006EEC0EF061C500F162C501F163C502F1D1
:103C500064C503F154EC26F004012C0E826F6EEC67
:103C60000EF078EC0EF039EF26F083C32AF184C30E
:103C70002BF185C32CF186C32DF187C32EF188C3A8
:103C80002FF189C330F18AC331F18BC332F18CC378
:103C900033F1010147EC2DF0BEEC2CF0160E0C6E4A
:103CA00000C10BF002EC0BF0170E0C6E01C10BF013
:103CB00002EC0BF0180E0C6E02C10BF002EC0BF0D4
:103CC000190E0C6E03C10BF002EC0BF000C18AF16F
:103CD00001C18BF102C18CF103C18DF100C18EF1E4
:103CE00001C18FF102C190F103C191F117EF1FF0F3
:103CF00083C32AF184C32BF185C32CF186C32DF134
:103D000087C32EF188C32FF189C330F18AC331F103
:103D10008BC332F18CC333F1010147EC2DF0BEECC3
:103D20002CF000C18AF101C18BF102C18CF103C1F9
:103D30008DF100C18EF101C18FF102C190F103C17B
:103D400091F117EF1FF083C32AF184C32BF185C3D0
:103D50002CF186C32DF187C32EF188C32FF189C3BF
:103D600030F18AC331F18CC332F18DC333F10101DB
:103D700047EC2DF0BEEC2CF00101000E046F000E9C
:103D8000056F010E066F000E076F0FEC2CF01A0E78
:103D90000C6E00C10BF002EC0BF01B0E0C6E01C19F
:103DA0000BF002EC0BF01C0E0C6E02C10BF002ECDF
:103DB0000BF01D0E0C6E03C10BF002EC0BF000C1FA
:103DC00092F101C193F102C194F103C195F117EF92
:103DD0001FF083C32AF184C32BF185C32CF186C362
:103DE0002DF187C32EF188C32FF189C330F18AC327
:103DF00031F18CC332F18DC333F1010147EC2DF069
:103E0000BEEC2CF00101000E046F000E056F010ED8
:103E1000066F000E076F0FEC2CF000C192F101C18C
:103E200093F102C194F103C195F117EF1FF0160E43
:103E300019EC0BF0E8CF00F1170E19EC0BF0E8CFFE
:103E400001F1180E19EC0BF0E8CF02F1190E19EC84
:103E50000BF0E8CF03F19CEC2CF07FEC2AF004018E
:103E6000730E826F6EEC0EF004012C0E826F6EECFE
:103E70000EF08AC100F18BC101F18CC102F18DC13C
:103E800003F19CEC2CF07FEC2AF00401730E826F9E
:103E90006EEC0EF004012C0E826F6EEC0EF01A0E1A
:103EA00019EC0BF0E8CF00F11B0E19EC0BF0E8CF8A
:103EB00001F11C0E19EC0BF0E8CF02F11D0E19EC0C
:103EC0000BF0E8CF03F154EC26F004012C0E826FC6
:103ED0006EEC0EF092C100F193C101F194C102F1B8
:103EE00095C103F154EC26F078EC0EF039EF26F092
:103EF0000401690E826F6EEC0EF004012C0E826FCD
:103F00006EEC0EF00101040E006F000E016F000E4A
:103F1000026F000E036F9CEC2CF02CC182F40401A4
:103F2000300E82276EEC0EF02DC182F40401300EAB
:103F300082276EEC0EF02EC182F40401300E82272F
:103F40006EEC0EF02FC182F40401300E82276EEC6D
:103F50000EF030C182F40401300E82276EEC0EF0B8
:103F600031C182F40401300E82276EEC0EF032C1B2
:103F700082F40401300E82276EEC0EF033C182F41D
:103F80000401300E82276EEC0EF004012C0E826FBD
:103F90006EEC0EF00101060E006F000E016F000EB8
:103FA000026F000E036F9CEC2CF02CC182F4040114
:103FB000300E82276EEC0EF02DC182F40401300E1B
:103FC00082276EEC0EF02EC182F40401300E82279F
:103FD0006EEC0EF02FC182F40401300E82276EECDD
:103FE0000EF030C182F40401300E82276EEC0EF028
:103FF00031C182F40401300E82276EEC0EF032C122
:1040000082F40401300E82276EEC0EF033C182F48C
:104010000401300E82276EEC0EF004012C0E826F2C
:104020006EEC0EF00101300E006F000E016F000EFD
:10403000026F000E036F9CEC2CF02CC182F4040183
:10404000300E82276EEC0EF02DC182F40401300E8A
:1040500082276EEC0EF02EC182F40401300E82270E
:104060006EEC0EF02FC182F40401300E82276EEC4C
:104070000EF030C182F40401300E82276EEC0EF097
:1040800031C182F40401300E82276EEC0EF032C191
:1040900082F40401300E82276EEC0EF033C182F4FC
:1040A0000401300E82276EEC0EF004012C0E826F9C
:1040B0006EEC0EF0200EF86EF76AF66A0401090045
:1040C000F5CF82F46EEC0EF00900F5CF82F46EECC1
:1040D0000EF00900F5CF82F46EEC0EF00900F5CF7A
:1040E00082F46EEC0EF00900F5CF82F46EEC0EF067
:1040F0000900F5CF82F46EEC0EF00900F5CF82F4E2
:104100006EEC0EF00900F5CF82F46EEC0EF078EC58
:104110000EF039EF26F08351630AD8A437EF26F06A
:104120008451610AD8A437EF26F085516C0AD8A4CF
:1041300037EF26F08651410A3FE08651440A1BE0E2
:104140008651420AD8B4EFEF20F08651350AD8B430
:10415000C3EF27F08651360AD8B418EF28F08651FD
:10416000370AD8B481EF28F08651380AD8B4DFEF87
:1041700028F037EF26F00798079A04017A0E826F2D
:104180006EEC0EF00401780E826F6EEC0EF00401FE
:10419000640E826F6EEC0EF00401550E826F6EECB1
:1041A0000EF0D8EF20F004014C0E826F6EEC0EF092
:1041B00078EC0EF039EF26F00788079A04017A0EA2
:1041C000826F6EEC0EF00401410E826F6EEC0EF009
:1041D0000401610E826F6EEC0EF0CCEF20F00798B8
:1041E000078A04017A0E826F6EEC0EF00401420E13
:1041F000826F6EEC0EF00401610E826F6EEC0EF0B9
:10420000CCEF20F0010166670DEF21F067670DEF3D
:1042100021F068670DEF21F0696715D04F6718EF3F
:1042200021F0506718EF21F0516718EF21F0526725
:104230000AD00101000E006F000E016F000E026F28
:10424000000E036F120011B80AD00101620E046F54
:10425000010E056F000E066F000E076F09D00101F9
:10426000A70E046F020E056F000E066F000E076F9B
:1042700066C100F167C101F168C102F169C103F1D2
:10428000FEEC2BF003BFB5EF21F0119A119C010158
:10429000000E046FA80E056F550E066F020E076F15
:1042A00066C100F167C101F168C102F169C103F1A2
:1042B00066C186F167C187F168C188F169C189F17A
:1042C000FEEC2BF003BF0BD00101000E866FA80E91
:1042D000876F550E886F020E896F118A119C0E0E22
:1042E00019EC0BF0E8CF18F10F0E19EC0BF0E8CF3A
:1042F00019F1100E19EC0BF0E8CF1AF1110E19ECB0
:104300000BF0E8CF1BF147EC2BF086C104F187C11D
:1043100005F188C106F189C107F1FEEC2BF0078297
:104320000BEC2BF047EC2BF007920BEC2BF086C13B
:1043300000F187C101F188C102F189C103F107923F
:104340000BEC2BF0CC0E046FE00E056F870E066FA2
:10435000050E076FFEEC2BF000C118F101C119F139
:1043600002C11AF103C11BF13BD0119C119A01014A
:10437000800E006F1A0E016F060E026F000E036FA3
:104380004FC104F150C105F151C106F152C107F10D
:10439000FEEC2BF003AF05D0F9EC2CF0118C119A48
:1043A00012000E0E19EC0BF0E8CF18F10F0E19ECFD
:1043B0000BF0E8CF19F1100E19EC0BF0E8CF1AF161
:1043C000110E19EC0BF0E8CF1BF14FC100F150C1F9
:1043D00001F151C102F152C103F107820BEC2BF044
:1043E00018C100F119C101F11AC102F11BC103F199
:1043F00012000401730E826F6EEC0EF004012C0E9D
:10440000826F6EEC0EF0078462C166F163C167F1E2
:1044100064C168F165C169F14BC14FF14CC150F104
:104420004DC151F14EC152F157C159F158C15AF124
:1044300007941FEC22F078EC0EF039EF26F066C1FD
:1044400000F167C101F168C102F169C103F1010125
:104450009CEC2CF07FEC2AF00401630E826F6EEC72
:104460000EF004012C0E826F6EEC0EF04FC100F1C5
:1044700050C101F151C102F152C103F101019CECA3
:104480002CF07FEC2AF00401660E826F6EEC0EF0C9
:1044900004012C0E826F6EEC0EF0F9EC2CF059C179
:1044A00000F15AC101F101019CEC2CF07FEC2AF0E3
:1044B0000401740E826F6EEC0EF012001082040183
:1044C000530E826F6EEC0EF004012C0E826F6EECB8
:1044D0000EF083C32AF184C32BF185C32CF186C36C
:1044E0002DF187C32EF188C32FF189C330F18AC320
:1044F00031F18BC332F18CC333F1010147EC2DF064
:10450000BEEC2CF000C166F101C167F102C168F197
:1045100003C169F18EC32AF18FC32BF190C32CF133
:1045200091C32DF192C32EF193C32FF194C330F1B7
:1045300095C331F196C332F197C333F1010147ECD2
:104540002DF0BEEC2CF000C14FF101C150F102C1C1
:1045500051F103C152F13AEC2DF099C32FF19AC3F6
:1045600030F19BC331F19CC332F19DC333F10101A2
:1045700047EC2DF0BEEC2CF000C159F101C15AF10D
:104580001FEC22F004012C0E826F6EEC0EF0D8EFBF
:1045900022F0118E19A002D019AE108C18BE02D0D4
:1045A00018A4108E8251520A02E10F8201D00F929C
:1045B0008251750A02E1108401D010948251550A8B
:1045C00002E1108601D0109611A003D011A401D0F1
:1045D0001084078410B246EF23F010A432EF23F0CA
:1045E000B6C166F1B7C167F1B8C168F1B9C169F187
:1045F000BAC16AF1BBC16BF1BCC16CF1BDC16DF157
:10460000BEC16EF1BFC16FF1C0C170F1C1C171F126
:10461000C2C172F1C3C173F1C4C174F1C5C175F1F6
:10462000C6C176F1C7C177F1C8C178F1C9C179F1C6
:10463000CAC17AF1CBC17BF1CCC17CF1CDC17DF196
:10464000CEC17EF1CFC17FF1D0C180F1D1C181F166
:10465000D2C182F1D3C183F1D4C184F1D5C185F136
:104660003AEF23F062C166F163C167F164C168F19A
:1046700065C169F14BC14FF14CC150F14DC151F1D0
:104680004EC152F157C159F158C15AF107940FA0C8
:1046900068EF23F00101926755EF23F0936755EF20
:1046A00023F0946755EF23F0956759EF23F068EFF7
:1046B00023F002EC21F092C104F193C105F194C101
:1046C00006F195C107F1FEEC2BF003BFFFEF25F0DB
:1046D00002EC21F00101000E046F000E056F010EC7
:1046E000066F000E076F2FEC2CF011A02CD011A23A
:1046F0002AD09CEC2CF0296701D007D004012D0EA4
:10470000826F6EEC0EF0FDEF25F030C182F40401F3
:10471000300E82276EEC0EF031C182F40401300EAF
:1047200082276EEC0EF032C182F40401300E822733
:104730006EEC0EF033C182F40401300E82276EEC71
:104740000EF0FDEF25F012A8C5D012981AC01BF08C
:104750001B3A1B42070E1B1600011B50000AD8B45F
:1047600036EF24F000011B50010AD8B4C2EF23F049
:1047700000011B50020AD8B4C0EF23F068EF24F008
:1047800068EF24F0F9EC2CF02AC001F12BC000F105
:10479000D89001330033D890013300330101630E08
:1047A000046F000E056F000E066F000E076F2FECF2
:1047B0002CF0280E046F000E056F000E066F000E21
:1047C000076FFEEC2BF000C12DF0F9EC2CF028C0A7
:1047D00001F1019F019D29C000F10101A40E046FA8
:1047E000000E056F000E066F000E076F2FEC2CF009
:1047F00000C12CF000C104F101C105F102C106F1B4
:1048000003C107F1640E006F000E016F000E026F0E
:10481000000E036FFEEC2BF0050E046F000E056F0B
:10482000000E066F000E076F2FEC2CF000C104F194
:1048300001C105F102C106F103C107F1F9EC2CF049
:104840002DC000F1FEEC2BF000C12EF02EC0E8FFD1
:10485000050F2D5C03E78A8468EF24F02EC0E8FF83
:104860000A0F2D5C01E68A9468EF24F000C124F160
:1048700001C125F102C126F103C127F1F9EC2CF0A9
:10488000FFEC2CF01A501F0BE8CF00F10101640E71
:10489000046F000E056F000E066F000E076F0FEC21
:1048A0002CF024C104F125C105F126C106F127C170
:1048B00007F1FEEC2BF003BF02D08A9401D08A846A
:1048C00024C100F125C101F126C102F127C103F184
:1048D000FFEF25F000C124F101C125F102C126F14D
:1048E00003C127F110AE4CD0109E00C108F101C1E8
:1048F00009F102C10AF103C10BF19CEC2CF030C1AB
:10490000D6F131C1D7F132C1D8F133C1D9F108C1E3
:1049100000F109C101F10AC102F10BC103F101016A
:104920006C0E046F070E056F000E066F000E076F0A
:10493000FEEC2BF003BF04D00101550EDA6F1CD042
:1049400008C100F109C101F10AC102F10BC103F173
:104950000101A40E046F060E056F000E066F000E17
:10496000076FFEEC2BF003BF04D001017F0EDA6F5E
:1049700003D00101FF0EDA6F1C8E11AEFFEF25F0A0
:1049800024C100F125C101F126C102F127C103F1C3
:1049900010A4D2EF24F00401750E826F6EEC0EF0BD
:1049A000D7EF24F00401720E826F6EEC0EF004015A
:1049B0002C0E826F6EEC0EF09CEC2CF02967E6EF6B
:1049C00024F00401200E826FE9EF24F004012D0E83
:1049D000826F6EEC0EF030C182F40401300E82273B
:1049E0006EEC0EF031C182F40401300E82276EECC1
:1049F0000EF004012E0E826F6EEC0EF032C182F4C6
:104A00000401300E82276EEC0EF033C182F40401F3
:104A1000300E82276EEC0EF004016D0E826F6EEC8C
:104A20000EF004012C0E826F6EEC0EF04FC100F1FF
:104A300050C101F151C102F152C103F101019CECDD
:104A40002CF07FEC2AF00401480E826F6EEC0EF021
:104A500004017A0E826F6EEC0EF004012C0E826F50
:104A60006EEC0EF066C100F167C101F168C102F1A0
:104A700069C103F101019CEC2CF07FEC2AF00401E8
:104A8000630E826F6EEC0EF004012C0E826F6EECE2
:104A90000EF066C100F167C101F168C102F169C1A0
:104AA00003F101010A0E046F000E056F000E066F80
:104AB000000E076F0FEC2CF0000E046F120E056F46
:104AC000000E066F000E076F2FEC2CF09CEC2CF004
:104AD0002AC182F40401300E82276EEC0EF02BC145
:104AE00082F40401300E82276EEC0EF02CC182F4A9
:104AF0000401300E82276EEC0EF02DC182F4040109
:104B0000300E82276EEC0EF02EC182F40401300EBE
:104B100082276EEC0EF02FC182F40401300E822742
:104B20006EEC0EF030C182F40401300E82276EEC80
:104B30000EF004012E0E826F6EEC0EF031C182F485
:104B40000401300E82276EEC0EF032C182F40401B3
:104B5000300E82276EEC0EF033C182F40401300E69
:104B600082276EEC0EF00401730E826F6EEC0EF075
:104B700004012C0E826F6EEC0EF0F9EC2CF059C192
:104B800000F15AC101F163EC27F00FB2CBEF25F031
:104B90000FA0FDEF25F004012C0E826F6EEC0EF0DD
:104BA000200EF86EF76AF66A04010900F5CF82F468
:104BB0006EEC0EF00900F5CF82F46EEC0EF00900F9
:104BC000F5CF82F46EEC0EF00900F5CF82F46EECB6
:104BD0000EF00900F5CF82F46EEC0EF00900F5CF6F
:104BE00082F46EEC0EF00900F5CF82F46EEC0EF05C
:104BF0000900F5CF82F46EEC0EF078EC0EF00F9019
:104C000039EF26F00401630E826F6EEC0EF00401A2
:104C10002C0E826F6EEC0EF03FEC26F004012C0E91
:104C2000826F6EEC0EF0B2EC26F004012C0E826F57
:104C30006EEC0EF02EEC27F004012C0E826F6EEC61
:104C40000EF00101F80E006FCD0E016F660E026FBF
:104C5000030E036F54EC26F004012C0E826F6EECF1
:104C60000EF044EC27F078EC0EF039EF26F078ECFB
:104C70000EF00301C26B0790109248EF29F0D89014
:104C80000E0E19EC0BF0E8CF00F10F0E19EC0BF043
:104C9000E8CF01F1100E19EC0BF0E8CF02F1110E84
:104CA00019EC0BF0E8CF03F10101000E046F000EC8
:104CB000056F010E066F000E076F2FEC2CF09CECB9
:104CC0002CF02AC182F40401300E82276EEC0EF023
:104CD0002BC182F40401300E82276EEC0EF02CC141
:104CE00082F40401300E82276EEC0EF02DC182F4A6
:104CF0000401300E82276EEC0EF02EC182F4040106
:104D0000300E82276EEC0EF02FC182F40401300EBB
:104D100082276EEC0EF030C182F40401300E82273F
:104D20006EEC0EF031C182F40401300E82276EEC7D
:104D30000EF004012E0E826F6EEC0EF032C182F482
:104D40000401300E82276EEC0EF033C182F40401B0
:104D5000300E82276EEC0EF004016D0E826F6EEC49
:104D60000EF01200120E19EC0BF0E8CF00F1130E4A
:104D700019EC0BF0E8CF01F1140E19EC0BF0E8CFB1
:104D800002F1150E19EC0BF0E8CF03F101010A0E48
:104D9000046F000E056F000E066F000E076F0FEC1C
:104DA0002CF0000E046F120E056F000E066F000E41
:104DB000076F2FEC2CF09CEC2CF02AC182F404013C
:104DC000300E82276EEC0EF02BC182F40401300EFF
:104DD00082276EEC0EF02CC182F40401300E822783
:104DE0006EEC0EF02DC182F40401300E82276EECC1
:104DF0000EF02EC182F40401300E82276EEC0EF00C
:104E00002FC182F40401300E82276EEC0EF030C107
:104E100082F40401300E82276EEC0EF004012E0E97
:104E2000826F6EEC0EF031C182F40401300E8227E5
:104E30006EEC0EF032C182F40401300E82276EEC6B
:104E40000EF033C182F40401300E82276EEC0EF0B6
:104E50000401730E826F6EEC0EF012000A0E19EC54
:104E60000BF0E8CF00F10B0E19EC0BF0E8CF01F1DD
:104E70000C0E19EC0BF0E8CF02F10D0E19EC0BF053
:104E8000E8CF03F163EF27F0060E19EC0BF0E8CF43
:104E900000F1070E19EC0BF0E8CF01F1080E19EC48
:104EA0000BF0E8CF02F1090E19EC0BF0E8CF03F19B
:104EB00063EF27F00101F9EC2CF0078457C100F1F2
:104EC00058C101F107940101E80E046F800E056FCF
:104ED000000E066F000E076F0FEC2CF0000E046F33
:104EE000040E056F000E066F000E076F2FEC2CF0FE
:104EF000880E046F130E056F000E066F000E076F0D
:104F0000FEEC2BF00A0E046F000E056F000E066F0C
:104F1000000E076F2FEC2CF09CEC2CF001012967A0
:104F200097EF27F00401200E826F9AEF27F004011B
:104F30002D0E826F6EEC0EF030C182F40401300E43
:104F400082276EEC0EF031C182F40401300E82270C
:104F50006EEC0EF032C182F40401300E82276EEC4A
:104F60000EF004012E0E826F6EEC0EF033C182F44F
:104F70000401300E82276EEC0EF00401430E826FA6
:104F80006EEC0EF0120087C32AF188C32BF189C39F
:104F90002CF18AC32DF18BC32EF18CC32FF18DC35D
:104FA00030F18EC331F190C332F191C333F101017D
:104FB000296B47EC2DF0BEEC2CF00101000E046FC4
:104FC000000E056F010E066F000E076F0FEC2CF040
:104FD0000E0E0C6E00C10BF002EC0BF00F0E0C6EFF
:104FE00001C10BF002EC0BF0100E0C6E02C10BF0C5
:104FF00002EC0BF0110E0C6E03C10BF002EC0BF087
:1050000004017A0E826F6EEC0EF004012C0E826F9A
:105010006EEC0EF00401350E826F6EEC0EF00401A2
:105020002C0E826F6EEC0EF03FEC26F0D8EF20F0E5
:1050300087C32AF188C32BF189C32CF18AC32DF1D0
:105040008BC32EF18CC32FF18DC330F18EC331F1A0
:1050500090C332F191C333F10101296B47EC2DF07C
:10506000BEEC2CF0880E046F130E056F000E066F59
:10507000000E076F03EC2CF0000E046F040E056F9A
:10508000000E066F000E076F0FEC2CF00101E80E0A
:10509000046F800E056F000E066F000E076F2FEC79
:1050A0002CF00A0E0C6E00C10BF002EC0BF00B0E94
:1050B0000C6E01C10BF002EC0BF00C0E0C6E02C179
:1050C0000BF002EC0BF00D0E0C6E03C10BF002ECBA
:1050D0000BF004017A0E826F6EEC0EF004012C0EC0
:1050E000826F6EEC0EF00401360E826F6EEC0EF0E5
:1050F00004012C0E826F6EEC0EF02EEC27F0D8EF30
:1051000020F087C32AF188C32BF189C32CF18AC30D
:105110002DF18BC32EF18CC32FF18DC330F18FC3D2
:1051200031F190C332F191C333F1010147EC2DF01D
:10513000BEEC2CF0000E046F120E056F000E066F11
:10514000000E076F0FEC2CF001010A0E046F000E29
:10515000056F000E066F000E076F2FEC2CF0120E7D
:105160000C6E00C10BF002EC0BF0130E0C6E01C1C3
:105170000BF002EC0BF0140E0C6E02C10BF002EC03
:105180000BF0150E0C6E03C10BF002EC0BF00401DA
:105190007A0E826F6EEC0EF004012C0E826F6EECB4
:1051A0000EF00401370E826F6EEC0EF004012C0E2F
:1051B000826F6EEC0EF0B2EC26F0D8EF20F087C3D1
:1051C0002AF188C32BF189C32CF18AC32DF18BC33B
:1051D0002EF18CC32FF18DC330F18EC331F190C30A
:1051E00032F191C333F10101296B47EC2DF0BEEC94
:1051F0002CF0880E046F130E056F000E066F000E64
:10520000076F03EC2CF0000E046F040E056F000E08
:10521000066F000E076F0FEC2CF00101E80E046F13
:10522000800E056F000E066F000E076F2FEC2CF03E
:10523000060E0C6E00C10BF002EC0BF0070E0C6EAC
:1052400001C10BF002EC0BF0080E0C6E02C10BF06A
:1052500002EC0BF0090E0C6E03C10BF002EC0BF02C
:1052600004017A0E826F6EEC0EF004012C0E826F38
:105270006EEC0EF00401380E826F6EEC0EF004013D
:105280002C0E826F6EEC0EF044EC27F0D8EF20F07D
:1052900007A8BBEF29F00101800E006F1A0E016F05
:1052A000060E026F000E036F4BC104F14CC105F1F5
:1052B0004DC106F14EC107F1FEEC2BF003BF01EF2B
:1052C0002AF079EC2AF04BC100F14CC101F14DC13B
:1052D00002F14EC103F107820BEC2BF018C104F16F
:1052E00019C105F11AC106F11BC107F1F80E006FD3
:1052F000CD0E016F660E026F030E036FFEEC2BF0F6
:105300000E0E0C6E00C10BF002EC0BF00F0E0C6ECB
:1053100001C10BF002EC0BF0100E0C6E02C10BF091
:1053200002EC0BF0110E0C6E03C10BF002EC0BF053
:1053300007840101F9EC2CF057C100F158C101F1CB
:1053400007940A0E0C6E00C10BF002EC0BF00B0E72
:105350000C6E01C10BF002EC0BF00C0E0C6E02C1D6
:105360000BF002EC0BF00D0E0C6E03C10BF002EC17
:105370000BF001EF2AF007AA01EF2AF007840101E0
:10538000F9EC2CF057C100F158C101F10794060E59
:105390000C6E00C10BF002EC0BF0070E0C6E01C19D
:1053A0000BF002EC0BF0080E0C6E02C10BF002ECDD
:1053B0000BF0090E0C6E03C10BF002EC0BF007842E
:1053C00062C100F163C101F164C102F165C103F181
:1053D0000794120E0C6E00C10BF002EC0BF0130ED2
:1053E0000C6E01C10BF002EC0BF0140E0C6E02C13E
:1053F0000BF002EC0BF0150E0C6E03C10BF002EC7F
:105400000BF00798079A0401805181197F0B0DE07A
:105410009EA8FED714EE00F081517F0BE126E750E5
:10542000812B0F01AD6E03EF2AF005012F51010A08
:1054300013E081AA2CEF2AF005012F51000A0AE09F
:105440000FB82CEF2AF0050130672CEF2AF00FB8C7
:105450002CEF2AF09BEF33F081B841EF2AF029ECD2
:105460002EF005012F51020A02E041EF2AF0602FD1
:1054700041EF2AF05FC560F50501010E306F3C0E6B
:10548000316FB5EF0DF018C100F119C101F11AC16A
:1054900002F11BC103F1000E046F000E056F010E37
:1054A000066F000E076F2FEC2CF029A16EEF2AF08B
:1054B0002051D8B46EEF2AF018C100F119C101F1E2
:1054C0001AC102F11BC103F1000E046F000E056F3B
:1054D0000A0E066F000E076F2FEC2CF01200010170
:1054E0000451001305510113065102130751031310
:1054F00012000101186B196B1A6B1B6B12002AC189
:1055000082F40401300E82276EEC0EF02BC182F47F
:105510000401300E82276EEC0EF02CC182F40401DF
:10552000300E82276EEC0EF02DC182F40401300E95
:1055300082276EEC0EF02EC182F40401300E822719
:105540006EEC0EF02FC182F40401300E82276EEC57
:105550000EF030C182F40401300E82276EEC0EF0A2
:1055600031C182F40401300E82276EEC0EF032C19C
:1055700082F40401300E82276EEC0EF033C182F407
:105580000401300E82276EEC0EF012002FC182F45F
:105590000401300E82276EEC0EF030C182F404015B
:1055A000300E82276EEC0EF031C182F40401300E11
:1055B00082276EEC0EF032C182F40401300E822795
:1055C0006EEC0EF033C182F40401300E82276EECD3
:1055D0000EF01200060E1E6E060E1F6E060E206ED8
:1055E0001E2EF0EF2AF01F2EF0EF2AF0202EF0EF03
:1055F0002AF08B84020E1E6E020E1F6E020E206EAB
:105600001E2E00EF2BF01F2E00EF2BF0202E00EFB0
:105610002BF08B9412000101005305E1015303E1CB
:10562000025301E1002BCEEC2BF0F9EC2CF03951B8
:10563000006F3A51016F420E046F4B0E056F000E62
:10564000066F000E076F0FEC2CF000C104F101C1D2
:1056500005F102C106F103C107F118C100F119C13A
:1056600001F11AC102F11BC103F107B23CEF2BF0AB
:1056700003EC2CF03EEF2BF0FEEC2BF000C118F108
:1056800001C119F102C11AF103C11BF11200F9ECB9
:105690002CF059C100F15AC101F1060E19EC0BF0C2
:1056A000E8CF04F1070E19EC0BF0E8CF05F1080E76
:1056B00019EC0BF0E8CF06F1090E19EC0BF0E8CF6E
:1056C00007F1FEEC2BF000C124F101C125F102C16C
:1056D00026F103C127F1290E046F000E056F000E9D
:1056E000066F000E076F0FEC2CF0EE0E046F430EEA
:1056F000056F000E066F000E076F03EC2CF024C13F
:1057000004F125C105F126C106F127C107F10FEC0F
:105710002CF000C11CF101C11DF102C11EF103C139
:105720001FF1120E19EC0BF0E8CF04F1130E19EC77
:105730000BF0E8CF05F1140E19EC0BF0E8CF06F1F1
:10574000150E19EC0BF0E8CF07F10D0E006F000EEF
:10575000016F000E026F000E036F0FEC2CF0180E9D
:10576000046F000E056F000E066F000E076F2FEC22
:105770002CF01CC104F11DC105F11EC106F11FC1B1
:1057800007F103EC2CF06A0E046F2A0E056F000E71
:10579000066F000E076FFEEC2BF01200BF0EFA6EC4
:1057A000200E3A6F396BD890003701370237033734
:1057B000D8B0DFEF2BF03A2FD4EF2BF039073A07B0
:1057C0000353D8B412000331070B80093F6F03392C
:1057D0000F0B010F396F80EC5FF0406F390580ECE3
:1057E0005FF0405D405F396B3F33D8B039273933C4
:1057F0003FA9F4EF2BF040513927120001011EECB4
:105800002DF0D8B01200010103510719346FE1ECFB
:105810002CF0D8900751031934AF800F120001010A
:10582000346B05EC2DF0D8A01BEC2DF0D8B0120095
:10583000F0EC2CF0F9EC2CF01F0E366F31EC2DF063
:105840000B35D8B0E1EC2CF0D8A00335D8B012005D
:10585000362F1EEF2CF034B108EC2DF012000101B0
:10586000346B04510511061107110008D8A005EC8E
:105870002DF0D8A01BEC2DF0D8B01200086B096BEE
:105880000A6B0B6B31EC2DF01F0E366F31EC2DF0E7
:1058900007510B5DD8A459EF2CF006510A5DD8A42E
:1058A00059EF2CF00551095DD8A459EF2CF00451A3
:1058B000085DD8A06CEF2CF00451085F0551D8A00A
:1058C000053D095F0651D8A0063D0A5F0751D8A0E3
:1058D000073D0B5FD8900081362F46EF2CF034B196
:1058E00008EC2DF0346B05EC2DF0D89035EC2DF054
:1058F00007510B5DD8A489EF2CF006510A5DD8A49E
:1059000089EF2CF00551095DD8A489EF2CF00451E2
:10591000085DD8A098EF2CF0003F98EF2CF0013FE5
:1059200098EF2CF0023F98EF2CF0032BD8B4120024
:1059300034B108EC2DF012000101346B05EC2DF0B0
:10594000D8B012003AEC2DF0200E366F0037013738
:105950000237033711EE33F00A0E376FE7360A0EBF
:10596000E75CD8B0E76EE552372FAEEF2CF0362F5C
:10597000A6EF2CF034B12981D890120001010A0E53
:10598000346F200E366F11EE29F03451376F0A0E46
:10599000D890E652D8B0E726E732372FC9EF2CF07F
:1059A0000333023301330033362FC3EF2CF0E750BB
:1059B000FF0FD8A00335D8B0120029B108EC2DF0A4
:1059C0001200045100270551D8B0053D01270651AA
:1059D000D8B0063D02270751D8B0073D0327120073
:1059E0000051086F0151096F02510A6F03510B6F8B
:1059F00012000101006B016B026B036B12000101CD
:105A0000046B056B066B076B12000335D8A0120000
:105A10000351800B001F011F021F031F003F18EFDF
:105A20002DF0013F18EF2DF0023F18EF2DF0032B62
:105A3000342B032512000735D8A012000751800B24
:105A4000041F051F061F071F043F2EEF2DF0053F03
:105A50002EEF2DF0063F2EEF2DF0072B342B0725D0
:105A600012000037013702370337083709370A3782
:105A70000B3712000101296B2A6B2B6B2C6B2D6BE2
:105A80002E6B2F6B306B316B326B336B120001015D
:105A90002A510F0B2A6F2B510F0B2B6F2C510F0B11
:105AA0002C6F2D510F0B2D6F2E510F0B2E6F2F5171
:105AB0000F0B2F6F30510F0B306F31510F0B316FB8
:105AC00032510F0B326F33510F0B336F120010A88E
:105AD00006D08994000EC76E220EC66E05D089844A
:105AE000000EC76E220EC66E050EE82EFED71200FF
:105AF00010A802D0898401D08994050EE82EFED723
:105B0000120067EC2DF09E96C69E000EC96EFF0E29
:105B10009EB602D0E82EFCD79E96C69E000EC96E99
:105B2000FF0E9EB602D0E82EFCD7C9CFAFF59E96E9
:105B3000C69E000EC96EFF0E9EB602D0E82EFCD7A0
:105B4000C9CFB0F59E96C69E000EC96EFF0E9EB6DA
:105B500002D0E82EFCD7C9CFB1F59E96C69E000EA6
:105B6000C96EFF0E9EB602D0E82EFCD7C9CFB2F5A3
:105B70009E96C69E000EC96EFF0E9EB602D0E82EFF
:105B8000FCD7C9CFB3F59E96C69E000EC96EFF0E18
:105B90009EB602D0E82EFCD7C9CFB4F59E96C69E1D
:105BA000000EC96EFF0E9EB602D0E82EFCD7C9CFFC
:105BB000B5F578EC2DF0120067EC2DF09E96C69EA0
:105BC000800EC96EFF0E9EB602D0E82EFCD79E96C0
:105BD000C69EAFC5C9FFFF0E9EB602D0E82EFCD709
:105BE0009E96C69EB0C5C9FFFF0E9EB602D0E82E97
:105BF000FCD79E96C69EB1C5C9FFFF0E9EB602D0C9
:105C0000E82EFCD79E96C69EB2C5C9FFFF0E9EB673
:105C100002D0E82EFCD79E96C69EB3C5C9FFFF0EE4
:105C20009EB602D0E82EFCD79E96C69EB4C5C9FF8C
:105C3000FF0E9EB602D0E82EFCD79E96C69EB5C536
:105C4000C9FFFF0E9EB602D0E82EFCD778EC2DF0EF
:105C5000120067EC2DF09E96C69E070EC96EFF0ED1
:105C60009EB602D0E82EFCD79E96C69E000EC96E48
:105C7000FF0E9EB602D0E82EFCD7C9CFAFF59E9698
:105C8000C69E000EC96EFF0E9EB602D0E82EFCD74F
:105C9000C9CFB0F59E96C69E000EC96EFF0E9EB689
:105CA00002D0E82EFCD7C9CFB1F59E96C69E000E55
:105CB000C96EFF0E9EB602D0E82EFCD7C9CFB2F552
:105CC00078EC2DF067EC2DF09E96C69E22C0C9FFA1
:105CD000FF0E9EB602D0E82EFCD79E96C69E000E02
:105CE000C96EFF0E9EB602D0E82EFCD7C9CFB6F51E
:105CF00078EC2DF0120067EC2DF09E96C69E870E74
:105D0000C96EFF0E9EB602D0E82EFCD79E96C69EA8
:105D1000AFC5C9FFFF0E9EB602D0E82EFCD79E96F7
:105D2000C69EB0C5C9FFFF0E9EB602D0E82EFCD7B6
:105D30009E96C69EB1C5C9FFFF0E9EB602D0E82E44
:105D4000FCD79E96C69EB2C5C9FFFF0E9EB602D076
:105D5000E82EFCD778EC2DF067EC2DF09E96C69ED1
:105D600023C0C9FFFF0E9EB602D0E82EFCD79E9638
:105D7000C69EB6C5C9FFFF0E9EB602D0E82EFCD760
:105D800078EC2DF0120067EC2DF09E96C69E870EE3
:105D9000C96EFF0E9EB602D0E82EFCD79E96C69E18
:105DA000000EC96EFF0E9EB602D0E82EFCD79E965E
:105DB000C69E800EC96EFF0E9EB602D0E82EFCD79E
:105DC0009E96C69E800EC96EFF0E9EB602D0E82E2D
:105DD000FCD79E96C69E800EC96EFF0E9EB602D060
:105DE000E82EFCD778EC2DF0120067EC2DF09E9693
:105DF000C69E870EC96EFF0E9EB602D0E82EFCD757
:105E00009E96C69E000EC96EFF0E9EB602D0E82E6C
:105E1000FCD79E96C69E000EC96EFF0E9EB602D09F
:105E2000E82EFCD79E96C69E800EC96EFF0E9EB6CB
:105E300002D0E82EFCD79E96C69E800EC96EFF0E3D
:105E40009EB602D0E82EFCD778EC2DF0120010A8F8
:105E50002DD067EC2DF09E96C69E23C0C9FFFF0E85
:105E60009EB602D0E82EFCD79E96C69E450EC96E01
:105E7000FF0E9EB602D0E82EFCD778EC2DF067EC32
:105E80002DF09E96C69E8F0EC96EFF0E9EB602D056
:105E9000E82EFCD79E96C69E000EC96EFF0E9EB6DB
:105EA00002D0E82EFCD778EC2DF0120067EC2DF034
:105EB0009E96C69E23C0C9FFFF0E9EB602D0E82E56
:105EC000FCD79E96C69E010EC96EFF0E9EB602D0EE
:105ED000E82EFCD778EC2DF067EC2DF09E96C69E50
:105EE000910EC96EFF0E9EB602D0E82EFCD79E968C
:105EF000C69EA50EC96EFF0E9EB602D0E82EFCD738
:105F000078EC2DF0120067EC2DF09E96C69E23C013
:105F1000C9FFFF0E9EB602D0E82EFCD79E96C69E05
:105F2000810EC96EFF0E9EB602D0E82EFCD778EC2B
:105F30002DF0120067EC2DF09E96C69E23C0C9FF7F
:105F4000FF0E9EB602D0E82EFCD79E96C69E010E8E
:105F5000C96EFF0E9EB602D0E82EFCD778EC2DF06D
:105F6000120067EC2DF09E96C69E910EC96EFF0E34
:105F70009EB602D0E82EFCD79E96C69EA50EC96E90
:105F8000FF0E9EB602D0E82EFCD778EC2DF0120062
:105F900067EC2DF09E96C69E910EC96EFF0E9EB6C2
:105FA00002D0E82EFCD79E96C69E000EC96EFF0E4C
:105FB0009EB602D0E82EFCD778EC2DF01200050139
:105FC000256B266B276B286B899A400EC76E200EB7
:105FD000C66E9E96C69E030EC96EFF0E9EB602D07A
:105FE000E82EFCD79E96C69E27C5C9FFFF0E9EB61B
:105FF00002D0E82EFCD79E96C69E26C5C9FFFF0E8E
:106000009EB602D0E82EFCD79E96C69E25C5C9FF37
:10601000FF0E9EB602D0E82EFCD79E96C69EC952B1
:10602000FF0E9EB602D0E82EFCD7898A0F01C95018
:10603000FF0A01E1120005012E51130A05E00501D6
:106040002E51170A0CE012000501F00E256FFF0E0D
:10605000266F0F0E276F000E286F38EF30F0050106
:10606000F00E256FFF0E266FFF0E276F000E286FB4
:10607000899A400EC76E200EC66E9E96C69E030E6F
:10608000C96EFF0E9EB602D0E82EFCD79E96C69E25
:1060900027C5C9FFFF0E9EB602D0E82EFCD79E96FC
:1060A000C69E26C5C9FFFF0E9EB602D0E82EFCD7BD
:1060B0009E96C69E25C5C9FFFF0E9EB602D0E82E4D
:1060C000FCD79E96C69EC952FF0E9EB602D0E82E01
:1060D000FCD7898A0F01C950FF0A1DE005012E5126
:1060E000130A05E005012E51170A0BE01200050105
:1060F000000E256F000E266F100E276F000E286F02
:1061000012000501000E256F000E266F000E276F8E
:10611000010E286F12000501256B266B276B286B7B
:1061200005012E51130A05E005012E51170A0CE056
:1061300012000501000E216F000E226F080E236F62
:10614000000E246FADEF30F00501000E216F000E40
:10615000226F800E236F000E246F21C500F122C52F
:1061600001F123C502F124C503F125C504F126C5BB
:1061700005F127C506F128C507F16FEC2AF000C12B
:1061800025F501C126F502C127F503C128F5899A35
:10619000400EC76E200EC66E9E96C69E030EC96E3A
:1061A000FF0E9EB602D0E82EFCD79E96C69E27C54F
:1061B000C9FFFF0E9EB602D0E82EFCD79E96C69E63
:1061C00026C5C9FFFF0E9EB602D0E82EFCD79E96CC
:1061D000C69E25C5C9FFFF0E9EB602D0E82EFCD78D
:1061E0009E96C69EC952FF0E9EB602D0E82EFCD7E0
:1061F000898AC950FF0A08E104C125F505C126F5C1
:1062000006C127F507C128F5D890050124332333AB
:10621000223321332151F00B216F216717EF31F029
:10622000226717EF31F0236717EF31F02467ADEFE6
:1062300030F00501100E2527E86A2623E86A272397
:10624000E86A28231200E86A05012E51130A06E0C5
:1062500005012E51170A0BE0020E1200050128510C
:10626000000A03E12751F00B07E0010E12000501BF
:106270002851000A01E0010E120029C500F12AC5CB
:1062800001F12BC502F12CC503F125C504F126C58A
:1062900005F127C506F128C507F1FEEC2BF003BF79
:1062A000120023EC31F0D8A4B5EF31F0899A400EFA
:1062B000C76E200EC66E9E96C69E060EC96EFF0E57
:1062C0009EB602D0E82EFCD7898A899A9E96C69EF1
:1062D000020EC96EFF0E9EB602D0E82EFCD79E9627
:1062E000C69E27C5C9FFFF0E9EB602D0E82EFCD77A
:1062F0009E96C69E26C5C9FFFF0E9EB602D0E82E0A
:10630000FCD79E96C69E25C5C9FFFF0E9EB602D03D
:10631000E82EFCD79E96C69E000EC96EFF0E9EB656
:1063200002D0E82EFCD7898A899A9E96C69E050ED1
:10633000C96EFF0E9EB602D0E82EFCD79E96C69E72
:10634000C952FF0E9EB602D0E82EFCD7C9B09EEF10
:1063500031F0898A0501100E2527E86A2623E86AAC
:106360002723E86A28233DEF31F01200899A400E76
:10637000C76E200EC66E9E96C69E060EC96EFF0E96
:106380009EB602D0E82EFCD7898A899A9E96C69E30
:10639000C70EC96EFF0E9EB602D0E82EFCD7898AC2
:1063A0000501256B266B276B286B1200899A400E1E
:1063B000C76E200EC66E9E96C69E050EC96EFF0E57
:1063C0009EB602D0E82EFCD79E96C69EC952FF0EFE
:1063D0009EB602D0E82EFCD7C9CF37F5898A1200C5
:1063E000899A400EC76E200EC66E9E96C69EB90E46
:1063F000C96EFF0E9EB602D0E82EFCD7898A120025
:10640000899A400EC76E200EC66E9E96C69EAB0E33
:10641000C96EFF0E9EB602D0E82EFCD7898AFF0E09
:10642000E82EFED7120023EC31F0D8A41200899A8E
:10643000400EC76E200EC66E9E96C69E030EC96E97
:10644000FF0E9EB602D0E82EFCD79E96C69E27C5AC
:10645000C9FFFF0E9EB602D0E82EFCD79E96C69EC0
:1064600026C5C9FFFF0E9EB602D0E82EFCD79E9629
:10647000C69E25C5C9FFFF0E9EB602D0E82EFCD7EA
:106480009E96C69EC952FF0E9EB602D0E82EFCD73D
:10649000898A0F01C950FF0AD8A40EEF33F0050115
:1064A000FE0E376F81EC2DF0AFC538F5B0C539F56C
:1064B000B1C53AF5B2C53BF5B3C53CF5B4C53DF53C
:1064C000B5C53EF50784B6C166F1B7C167F1B8C17D
:1064D00068F1B9C169F14BC14FF14CC150F14DC1E7
:1064E00051F14EC152F157C159F158C15AF102EC64
:1064F00021F000C13FF501C140F502C141F503C1E2
:1065000042F5050161678CEF32F062678CEF32F083
:1065100063678CEF32F0646790EF32F09DEF32F0FA
:1065200061C504F162C505F163C506F164C507F1F3
:10653000FEEC2BF003BF0EEF33F059C143F55AC107
:1065400044F5B9C545F5BAC546F507940501110EE0
:10655000326F899A400EC76E200EC66E9E96C69EFA
:10656000060EC96EFF0E9EB602D0E82EFCD7898AB1
:10657000899A9E96C69E020EC96EFF0E9EB602D0E6
:10658000E82EFCD79E96C69E27C5C9FFFF0E9EB675
:1065900002D0E82EFCD79E96C69E26C5C9FFFF0EE8
:1065A0009EB602D0E82EFCD79E96C69E25C5C9FF92
:1065B000FF0E9EB602D0E82EFCD725EE37F0322F24
:1065C00002D0EEEF32F09E96C69EDECFC9FFFF0EE0
:1065D0009EB602D0E82EFCD7DFEF32F0898A899A86
:1065E0009E96C69E050EC96EFF0E9EB602D0E82E80
:1065F000FCD79E96C69EC952FF0E9EB602D0E82ECC
:10660000FCD7C9B0F9EF32F0898A0501100E2527B1
:10661000E86A2623E86A2723E86A2823120021C5AE
:1066200000F122C501F123C502F124C503F1899AC5
:10663000400EC76E200EC66E9E96C69E0B0EC96E8D
:10664000FF0E9EB602D0E82EFCD79E96C69E02C1D3
:10665000C9FFFF0E9EB602D0E82EFCD79E96C69EBE
:1066600001C1C9FFFF0E9EB602D0E82EFCD79E9650
:10667000C69E00C1C9FFFF0E9EB602D0E82EFCD711
:106680009E96C69EC952FF0E9EB602D0E82EFCD73B
:1066900025EE37F00501100E326F9E96C69EC95248
:1066A000FF0E9EB602D0E82EFCD7C9CFDEFF322FF8
:1066B0004DEF33F0898A1200899A400EC76E200E82
:1066C000C66E9E96C69E900EC96EFF0E9EB602D0F6
:1066D000E82EFCD79E96C69E000EC96EFF0E9EB693
:1066E00002D0E82EFCD79E96C69E000EC96EFF0E05
:1066F0009EB602D0E82EFCD79E96C69E000EC96EAE
:10670000FF0E9EB602D0E82EFCD79E96C69EC952BA
:10671000FF0E9EB602D0E82EFCD7C9CF2DF59E966F
:10672000C69EC952FF0E9EB602D0E82EFCD7C9CF36
:106730002EF5898A1200EAEC2AF0B9C5E8FFD708DD
:1067400002E3EAEC2AF0B9C5E8FFC80802E3EAEC84
:106750002AF0B9C5E8FFB90802E3EAEC2AF0B9C5A6
:10676000E8FFAA0802E3EAEC2AF0B9C5E8FF9B08B3
:1067700002E3EAEC2AF029EC2EF0F0EC31F0F29C86
:10678000F29E8B94C69AC2909482948C720ED36EB1
:10679000D3A4FED789968A909390FF0EE8CF00F09D
:1067A000E82EFED7002EFCD78150F294F29A9E90EC
:1067B0009D909E929D92F298F292F290F286F28EC5
:0467C0000300FF00D3
:10BF0000E844F926000C160C2B0C3F0C520C640C68
:10BF1000760C860C960CA50CB30CC10CCF0CDC0C6B
:06BF2000E80CF40C000C1B
:0200000400F00A
:0100C800FE39
:00000001FF
